:100000000C94B7010C94E2310C940F320C94DF0184
:100010000C94DF010C94DF010C94DF010C94DF01E0
:100020000C94DF010C94DF010C94DF010C94CA06E0
:100030000C94DF010C94DF010C94DF010C94DF01C0
:100040000C94EE300C94DF010C9440060C947C066A
:100050000C94DF010C94DF010C94DF010C94DF01A0
:100060000C94DF010C94DF01084AD73B3BCE016EB4
:1000700084BCBFFDC12F3D6C74319ABD56833DDAFF
:100080003D00C77F11BED9E4BB4C3E916BAAAABE0E
:10009000000000803F05A84CCDB2D44EB93836A937
:1000A000020C50B9918688083CA6AAAA2ABE000074
:1000B00000803F0664EC1B3C04BC163E3BE5B93CAB
:1000C000C93C37C29E5A3D660498083EEA69AAAA0E
:1000D0003E000000803F2020BF0020BF00BF007C0A
:1000E0002020202020202020202020202020202010
:1000F00020202000C8202020202020202020202078
:1001000020C900C8202020202020202020202020BE
:10011000C97C00D820202020202020202020202042
:10012000D97C00C820202020202020202020202032
:10013000C97C00C820202020202020202020202032
:10014000C97C00207265766F006D696E6F706F7389
:1001500064206C6962726570696C6F740020202085
:100160002020BABBBCBDBE7C2020202020CACBCC26
:10017000CDCE7C00626F6F74696E672075703AED4A
:10018000F2F2F2F2F2F2F2F30062617474657279E3
:10019000207761726E696E672000747870696420E0
:1001A00076616C756573006261726F2074656D7045
:1001B0000074656D706469737020006163746976A2
:1001C000652000706173736976650075617674618E
:1001D0006C6B200073657475702073637265656E57
:1001E0007C7C7C004368617220446F6E650A00521B
:1001F0006561647920666F7220466F6E740A0055DF
:1002000070646174652043686172536574000040D6
:100210007A10F35A00A0724E18090010A5D4E80015
:1002200000E87648170000E40B54020000CA9A3B2D
:10023000000000E1F50500008096980000004042B3
:100240000F000000A0860100000010270000000041
:10025000E803000000006400000000000A00000045
:1002600000000100000000002C76D888DC674F08F1
:1002700023DFC1DFAE59E1B1B796E5E3E453C63AF7
:10028000E651997696E8E6C28426EB898C9B62ED6E
:10029000407C6FFCEFBC9C9F40F2BAA56FA5F49028
:1002A000055A2AF75C936B6CF9676DC11BFCE0E49F
:1002B0000D47FEF520E6B500D0ED902E03009435F5
:1002C00077050080841E080000204E0A000000C848
:1002D0000C333333330F986E12831141EF8D211499
:1002E000893BE65516CFFEE6DB18D1844B381BF769
:1002F0007C1D901DA4BBE424203284725E22810008
:10030000C9F124ECA1E53D276E616E00696E6600BF
:1003100000000000240027002A0000000000250043
:1003200028002B0000000000230026002900040400
:10033000040404040404020202020202030303038D
:100340000303010204081020408001020408102069
:100350000102040810200000000700020100000351
:10036000040600000000000000004B0411081124E6
:100370001FBECFEFD8E0DEBFCDBF14E0A0E0B1E0FC
:10038000ECE6FEE602C005900D92AA30B107D9F75F
:1003900016E0AAE0B4E001C01D92AC3BB107E1F762
:1003A00013E0CEE6D3E004C02297FE010E9430376E
:1003B000CA36D107C9F70E94F9320C9434370C942D
:1003C0000000FA01AA27283051F1203181F1E89488
:1003D0006F936E7F6E5F7F4F8F4F9F4FAF4FB1E038
:1003E0003ED0B4E03CD0670F781F891F9A1FA11D33
:1003F000680F791F8A1F911DA11D6A0F711D811D34
:10040000911DA11D20D009F468943F912AE0269FF8
:1004100011243019305D3193DEF6CF010895462F57
:100420004770405D4193B3E00FD0C9F7F6CF462F38
:100430004F70405D4A3318F0495D31FD40524193A1
:1004400002D0A9F7EACFB4E0A6959795879577955E
:100450006795BA95C9F700976105710508959B01E5
:10046000AC010A2E06945795479537952795BA956E
:10047000C9F7620F731F841F951FA01D08952830B0
:1004800008F027E03327DA01990F311D87FD9160CD
:1004900000966105710539F432602E5F3D9330E3BB
:1004A0002A95E1F708959F3F30F080387105610586
:1004B00009F03C5F3C5F3D93913008F08068911DEE
:1004C000DF93CF931F930F93FF92EF92192F987F93
:1004D0009695E92F96959695E90FFF27E859FD4FD8
:1004E00099273327EE24FF24A701E70105900894FC
:1004F000079428F4360FE71EF81E491F511D660F9A
:10050000771F881F991F0694A1F70590079428F478
:10051000E70EF81E491F561FC11D770F881F991F30
:10052000661F0694A1F70590079428F4F80E491F5A
:10053000561FC71FD11D880F991F661F771F06946E
:10054000A1F70590079420F4490F561FC71FD81F25
:10055000990F661F771F881F0694A9F7849110953D
:10056000177041F0D695C79557954795F794E7943E
:100570001A95C1F7EEE0F2E0689415901591359167
:100580006591959105907FE27395E118F10A430B0F
:10059000560BC90BD009C0F7E10CF11E431F561FC3
:1005A000C91FD01D7EF4703311F48A95E6CFE8940C
:1005B000015030F0080F0AF40027021708F4202F2A
:1005C0002395022F7A3328F079E37D932A95E9F772
:1005D00010C07D932A9589F606949795679537956F
:1005E00017951794E118F10A430B560BC90BD00964
:1005F00098F023957E9173957A3308F070E37C939D
:100600002013B8F77E9170617D9330F0839571E38C
:100610007D9370E32A95E1F71124EF90FF900F91FD
:100620001F91CF91DF91992787FD90950895CF93E2
:10063000DF93BC018230910510F462E070E0A0917C
:10064000BA06B091BB06ED0140E050E0E0E0F0E01A
:1006500021C0888199818617970769F48A819B81D7
:10066000309719F09383828304C09093BB068093E4
:10067000BA06FE0134C06817790738F441155105F0
:1006800019F08417950708F4AC01FE018A819B815B
:100690009C01E9012097E9F641155105A9F1CA012C
:1006A000861B970B049708F4BA01E0E0F0E02AC03B
:1006B0008D919C91119784179507F9F4641775072C
:1006C00081F412968D919C911397309719F0938332
:1006D000828304C09093BB068093BA06FD013296D4
:1006E0004CC0CA01861B970BFD01E80FF91F6193EF
:1006F000719302978D939C9340C0FD0182819381F9
:100700009C01D9011097A1F68091B8069091B90685
:10071000892B41F48091AC029091AD029093B9067F
:100720008093B8064091AE025091AF024115510539
:1007300041F44DB75EB78091AA029091AB02481B7D
:10074000590B2091B8063091B906CA01821B930B50
:100750008617970780F0AB014E5F5F4F84179507B0
:1007600050F0420F531F5093B9064093B806F90159
:100770006193719302C0E0E0F0E0CF01DF91CF918F
:100780000895CF93DF93009709F450C0EC012297AE
:100790001B821A82A091BA06B091BB06109709F18C
:1007A00040E050E0AC17BD0708F1BB83AA83FE010F
:1007B00021913191E20FF31FAE17BF0779F48D91AC
:1007C0009C911197280F391F2E5F3F4F3983288343
:1007D00012968D919C9113979B838A8341155105A5
:1007E00071F4D093BB06C093BA0620C012968D91C7
:1007F0009C911397AD01009711F0DC01D3CFFA0162
:10080000D383C28321913191E20FF31FCE17DF070B
:1008100069F488819981280F391F2E5F3F4FFA01B3
:10082000318320838A819B8193838283DF91CF915F
:100830000895FC010590615070400110D8F7809533
:1008400090958E0F9F1F0895FC016150704001909C
:100850000110D8F7809590958E0F9F1F08956EBD5B
:100860000DB407FEFDCF8EB508958DE061E00E94C6
:100870003C328BE061E00E943C328CE060E00E9400
:100880003C328AE061E00E943C321CBC80E58CBDB9
:100890008DB58EB508958AE094E00E9435040895E0
:1008A000FC011382128288EE93E0A0E0B0E0848322
:1008B0009583A683B78380EC92E09183808308952B
:1008C000FC018089803419F421E030E002C020E08E
:1008D00030E0C9010895FC01818990E00895FC0190
:1008E0006487458766874787089580E090E008958C
:1008F00080E090E0089580E090E008950895EF9200
:10090000FF921F93CF93DF93162F7A0186E060E06A
:100910000E947B328AE094E060E00E942F048AE02B
:1009200094E060E00E942F048AE094E069E00E9475
:100930002F048AE094E0612F0E942F04C0E0D0E0F1
:10094000F701EC0FFD1F10818AE094E06AE00E943D
:100950002F048AE094E06C2F0E942F048AE094E038
:100960006BE00E942F048AE094E0612F0E942F0424
:100970002196C633D10521F78AE094E068E00E9411
:100980002F048AE094E060EA0E942F048AE094E059
:1009900060EA0E942F0485FDF9CF8AE094E060E0D0
:1009A0000E942F048AE094E06CE00E942F0486E00D
:1009B00061E00E947B32DF91CF911F91FF90EF9019
:1009C00008951F93CF93DF93EC01162F86E060E02C
:1009D0000E947B328AE094E060E00E942F041123A1
:1009E00019F0113059F404C08AE094E0688904C019
:1009F00068896C618AE094E00E942F0486E061E0DF
:100A00000E947B32DF91CF911F910895EF92FF9268
:100A10000F931F938EE1489F70011124E60EF11C85
:100A200086E060E00E947B320AE014E0C80165E0E5
:100A30000E942F04C8016F2D0E942F04C80166E098
:100A40000E942F04C8016E2D0E942F041F910F9148
:100A5000FF90EF900895EF92FF920F931F937C0108
:100A60000AE014E0C80167E00E942F04C8016FEF9C
:100A70000E942F0486E061E00E947B32F7018785A7
:100A80008F5F87871F910F91FF90EF900895EF92EE
:100A9000FF920F931F93FC01E7848EE1E89E7001A3
:100AA00011248685E80EF11C86E060E00E947B320E
:100AB0000AE014E0C80164E00E942F04C80163E06A
:100AC0000E942F04C80165E00E942F04C8016F2D09
:100AD0000E942F04C80166E00E942F04C8016E2DF9
:100AE0000E942F041F910F91FF90EF9008951F9384
:100AF000CF93DF93EC01162F6C3731F40E942B0556
:100B0000CE010E9447050AC08AE094E067E00E9497
:100B10002F048AE094E0612F0E942F0481E090E08E
:100B2000DF91CF911F9108950F931F9386E060E0AE
:100B30000E947B320AE014E0C80164E00E942F04A6
:100B4000C80164E00E942F0486E061E00E947B32CD
:100B50001F910F9108951F93CF93DF93EC01188A93
:100B600016E0198B88EA96E060E973E00E944E3047
:100B7000813049F480E4888B88E0898B86E060E0EE
:100B80000E947B3202C0188A198B86E060E00E94C6
:100B90007B32DF91CF911F9108950F931F93CF93D5
:100BA000DF93EC0186E061E00E943C3282E060E08D
:100BB0000E943C3282E061E00E947B32CE010E94C2
:100BC000AB0586E060E00E947B328AE094E06CEE48
:100BD0000E942F048AE094E06FEF0E942F04182FE8
:100BE0008AE094E060E00E942F04688962608AE0F5
:100BF00094E00E942F0462E370E080E090E00E94A5
:100C000044318AE094E06CE60E942F041F7E8AE063
:100C100094E0612F0E942F048889803419F00DE040
:100C200010E002C000E110E010920C0410920B04DE
:100C300017C060910B0470910C04605F8AE094E02F
:100C40000E942F048AE094E069E00E942F048091C2
:100C50000B0490910C04019690930C0480930B0468
:100C600080910B0490910C048017910714F3CE012E
:100C700061E00E94E104DF91CF911F910F910895EF
:100C80001F920F920FB60F9211242F933F934F9301
:100C90008F939F93EF93FF934091C6002091970607
:100CA000309198062F5F3F4F80919B0690919C0654
:100CB000282339238091990690919A06281739079D
:100CC00079F08091970690919806E0919D06F091B9
:100CD0009E06E80FF91F40833093980620939706ED
:100CE000FF91EF919F918F914F913F912F910F9095
:100CF0000FBE0F901F9018951F920F920FB60F9274
:100D000011242F933F938F939F93EF93FF93209101
:100D1000A1063091A20680919F069091A006281707
:100D20003907E9F08091A1069091A206E091A5060D
:100D3000F091A606E80FF91F80818093C60080918C
:100D4000A1069091A20601962091A3063091A406D7
:100D5000822393239093A2068093A10610C0209132
:100D60009F063091A0068091A1069091A2062817B7
:100D7000390729F48091C1008F7D8093C100FF91D4
:100D8000EF919F918F913F912F910F900FBE0F90F8
:100D90001F9018951F920F920FB60F9211248F93E8
:100DA0009F938091CD049091CE04892B51F0809136
:100DB000CF049091D00401969093D0048093CF04F7
:100DC00009C08091D1049091D20401969093D204ED
:100DD0008093D1049F918F910F900FBE0F901F9021
:100DE0001895CF93DF93482FEB0180912E06833027
:100DF00009F45DC0843028F48130C1F0823058F5A8
:100E00000AC0853009F4D2C0853008F4A8C0863005
:100E100009F0F2C0E9C04C3309F0EEC081E08093E4
:100E20002E06488384EB80932D06E6C0842F90E045
:100E3000E0912D06F0E0E827F927E253FD4F2081ED
:100E400020932D06887F9070809741F582E08093F3
:100E50002E06498329C0242F30E0E0912D06F0E0D2
:100E6000E227F327E253FD4F808180932D06809186
:100E70002C068F5F80932C06823018F43B832A83E4
:100E8000BBC0922F88272A813B81820F931F9B83AF
:100E90008A830A978F3F910521F018F010922E0651
:100EA000ABC083E080932E0610922C06A5C0E42FE1
:100EB000F0E080912D0690E0E827F927E253FD4FFE
:100EC000808180932D0660912C066F5F60932C06C5
:100ED000623089F0633020F4613009F08DC006C0C3
:100EE000633091F0643009F087C022C0842F90E015
:100EF000A0E0B0E018C0242F30E040E050E0542FD4
:100F0000432F322F222707C0242F30E040E050E04B
:100F1000A901332722278C819D81AE81BF81820F59
:100F2000931FA41FB51F8C839D83AE83BF8364C0B2
:100F3000242F30E040E050E0522F4427332722276F
:100F40008C819D81AE81BF81820F931FA41FB51F2D
:100F50008C839D83AE83BF8360932E06A5CF242F01
:100F600030E0E0912D06F0E0E227F327E253FD4F59
:100F7000808180932D0680912C068F5F80932C06B4
:100F8000813019F08230C1F503C03987288734C019
:100F9000922F882728853985280F391F3987288778
:100FA0008A819B810A97F1F085E07CCFE42FF0E005
:100FB00080912D0690E0E827F927E253FD4F8081CC
:100FC00080932D0620912C062F5F20932C0630E075
:100FD000FB01E20FF31F41878A819B810A97281743
:100FE000390750F086E05ECFC75FDE4F4883C950B7
:100FF000D14087E080932E0680912E06873069F4D9
:1010000010922E06C75FDE4F90912D068881C95041
:10101000D140981711F48A8101C080E0DF91CF910F
:1010200008958F92AF92CF92EF92FF920F931F93FA
:1010300083E994E060E045EC50E024EC30E000EC23
:1010400010E0B1ECEB2EF12CCC24C394A8E9AA2E2D
:10105000F0E28F2E0E94BE2980EB94E00E945004A3
:101060001092C3041092C4041092C5041092C604D6
:101070001092C7041092C8041092C9041092CA04B6
:101080001092CC041092CB041092C2041F910F91C5
:10109000FF90EF90CF90AF908F900895AF92BF9256
:1010A000CF92DF92EF92FF920F931F93E0909306FF
:1010B000F090940600919506109196068FE590E0C9
:1010C000A0E0B0E0E80EF91E0A1F1B1F0E94363197
:1010D0006E157F058007910708F44EC0A090F804B4
:1010E000B090F904C090FA04D090FB04C601B50199
:1010F00020E030E040E85FE30E949935181694F54F
:10110000E0904B06F0904C0600914D0610914E0673
:101110000E943631209193063091940640919506B5
:1011200050919606621B730B840B950B0E946F34D3
:101130009B01AC01C601B5010E94A43520E030E05E
:101140004AE754E40E94D6339B01AC01C801B701C1
:101150000E94093360934B0670934C0680934D06B2
:1011600090934E060E9436316093930670939406D6
:1011700080939506909396061F910F91FF90EF90A4
:10118000DF90CF90BF90AF900895DF93CF9300D0C2
:1011900000D0CDB7DEB7FB01E80FF91F628583856C
:1011A0009485258569838A839B832C83492F5C8161
:1011B000782FCA010F900F900F900F90CF91DF9171
:1011C0000895AF92BF92DF92EF92FF920F931F9319
:1011D000CF93DF938C0180912F0680FDE4C0F8014E
:1011E000F08083E994E06F2D0E949F2AE801C75F99
:1011F000DE4FEF2DF0E0E253FD4F80818883F80150
:10120000F18083E994E06F2D0E949F2AEF2DF0E09A
:10121000888190E0E827F927E253FD4F8081888399
:10122000F801F28083E994E06F2D0E949F2AEF2D50
:10123000F0E0888190E0E827F927E253FD4F8081B4
:101240008883F801F38083E994E06F2D0E949F2A40
:10125000EF2DF0E0888190E0E827F927E253FD4F79
:1012600080818883F801F48083E994E06F2D0E94E7
:101270009F2AEF2DF0E0888190E0E827F927E253DC
:10128000FD4F80818883F801248135814681578113
:10129000232F342F452F5527F22E83E994E0622F18
:1012A0000E949F2AEF2DF0E0888190E0E827F9273F
:1012B000E253FD4F80818883F80124813581468186
:1012C00057819A0144275527F22E83E994E0622F33
:1012D0000E949F2AEF2DF0E0888190E0E827F9270F
:1012E000E253FD4F80818883F80124813581468156
:1012F0005781252F332744275527F22E83E994E081
:10130000622F0E949F2AEF2DF0E0888190E0E8276D
:10131000F927E253FD4F8081888383E994E060E000
:101320000E949F2AE881F0E0E253FD4F808188838C
:1013300083E994E060E00E949F2AE881F0E0E253B4
:10134000FD4F80818883F801828193810B9718F18A
:101350008AE0A82EB12CA00EB11E750112C0F701B3
:10136000D1907F0183E994E06D2D0E949F2AED2D9D
:10137000F0E0888190E0E827F927E253FD4F808173
:1013800088832E2D2A1930E0F801828193810A97F3
:101390002817390720F3075F1E4F83E994E0F8010F
:1013A00060810E949F2ADF91CF911F910F91FF9042
:1013B000EF90DF90BF90AF900895DF93CF93CDB7BC
:1013C000DEB7CA50D1400FB6F894DEBF0FBECDBF16
:1013D0002CE329836A832AE030E03C832B83FC01E1
:1013E00084819581A681B7818D839E83AF83B887E1
:1013F000CE0101960E94E108C65FDE4F0FB6F89459
:10140000DEBF0FBECDBFCF91DF91089588EA96E091
:101410006AE773E00E944E30882331F586E696E64F
:10142000A6E6B0E48093300690933106A09332068E
:10143000B093330680E090E0A0E8BFE380933406E9
:1014400090933506A0933606B093370688EE93E066
:10145000909339068093380681E880933A068DE8A8
:1014600080933B068DEF25C082E598EBAEE0B0E4BB
:101470008093300690933106A0933206B0933306E2
:1014800085E89BEEA1E5B0E48093340690933506A1
:10149000A0933606B093370680EA94E1909339061C
:1014A000809338068BEF80933A0686E680933B065E
:1014B0008AEF80933C060895FF920F931F9308EAEA
:1014C00016E0C8016CE773E00E944E308093770607
:1014D000C8016EE773E00E944E3080937806C80121
:1014E00060E873E00E944E3080935706C8016EE8B2
:1014F00073E00E944E3080936F06C8016AE873E083
:101500000E944E3080936D06C80164E873E00E942B
:101510004E3080937906C80166E873E00E944E3031
:1015200080937A06C8016CE873E00E944E30809385
:101530005F06C80162E973E00E944E3080937B062B
:10154000C80164E973E00E944E3080935E06C801D2
:1015500064EF73E00E944E30F82EC80165EF73E02F
:101560000E944E30382F20E02F0D311D30937D0624
:1015700020937C06C80166EF73E00E944E30F82E7F
:10158000C80167EF73E00E944E30382F20E02F0D26
:10159000311D30937F0620937E06C80168EF73E00B
:1015A0000E944E30F82EC80169EF73E00E944E3061
:1015B000382F20E02F0D311D3093810620938006B7
:1015C000C8016BEF73E00E944E30809356061F9166
:1015D0000F91FF900895BC0188EA96E00E944E307A
:1015E00008956091E2047091E3048091E404909185
:1015F000E50420E030E040E152E40E94A43520E020
:1016000030E044EB53E40E94D6330E9407360E9438
:101610003E349B012550304037FF03C09B01215EC3
:101620003F4FAFE3B6E0F901E253FC4F80818C936A
:101630002F5F3F4F2432310514F020E030E0119647
:1016400086E0AA34B80779F71C9208952F923F924A
:101650004F925F926F927F928F929F92AF92BF92C2
:10166000CF92DF92EF92FF920F931F93DF93CF936E
:1016700000D000D000D0CDB7DEB7182F662E209155
:10168000D8043091D9042A35310530F0C9018D5480
:101690009F4F89359105E8F437FF02C02D543F4F25
:1016A000C90137FF03C0909581959F4F8A319105FD
:1016B0003CF0F4E48F2E912CE9ED2E2E312C1DC040
:1016C0000A975CF17BE3872E912C62ED262E312C5C
:1016D00020C02B35310514F0235B3040C90137FFA2
:1016E00003C0909581959F4F8A31910554F056E53E
:1016F000852E912C4CED242E312C37E0A32EB12CCD
:1017000015C00A9754F02DE4822E912C94ED292EC9
:10171000312C88E0A82EB12C09C005E0802E912C38
:10172000B8E32B2E312CA9E0AA2EB12C6091DA045B
:101730007091DB04882777FD8095982F0E94713483
:1017400027EA32E94BE25CEB0E94A4350E9478362E
:1017500020E030E040EA50E40E94A43520E030E090
:1017600040E951E40E94A4350E94073620E030E0B1
:1017700044E352E40E9409330E943E34712EFEEB92
:10178000CF2EFFEFDF2E9B01442737FD4095542FCE
:1017900029833A834B835C83E0EB4E2EE4E05E2E9C
:1017A0004AEF5FEF240E351E6091D8047091D90482
:1017B000882777FD8095982F0E94713425E33AEFB2
:1017C0004EE85CE30E94A4350E9478367B018C01D0
:1017D000B601882777FD8095982F0E9471349B0170
:1017E000AC01C801B7010E94A4357B018C0169815D
:1017F0007A818B819C810E9471349B01AC01C8016C
:10180000B7010E9409330E943E349B01CB0101972E
:101810008A35910508F071C062E170E00E94DE3601
:101820008B012F5F3F4FAEEEBFEF6A9FC0016B9FF2
:10183000900D7A9F900D1124820F931F62E070E04B
:101840000E94DE366D837E83E62CE01A4E2D4C5FBF
:1018500080EB94E0672D0E94060500D000D000D0F8
:10186000EDB7FEB73196ADB7BEB712965C924E9209
:10187000119720E031E0338322838D819E81880D92
:10188000991D958384830E949D294DB75EB74A5F59
:101890005F4F0FB6F8945EBF0FBE4DBF8D819E8126
:1018A0008A159B0554F1043011053CF593E0E90ECF
:1018B000C201672D4E2D0E94060500D000D000D039
:1018C000EDB7FEB73196ADB7BEB712965C924E92A9
:1018D000119720E031E0338322834D815E81420DF8
:1018E000531D558344830E949D298DB79EB706964C
:1018F0000FB6F8949EBF0FBE8DBFACE0B0E0CA0E2D
:10190000DB1E7394BEE4CB16D10409F04DCF2696AE
:101910000FB6F894DEBF0FBECDBFCF91DF911F9100
:101920000F91FF90EF90DF90CF90BF90AF909F907E
:101930008F907F906F905F904F903F902F90089581
:10194000823010F422E002C0282F220F30E08DB741
:101950009EB708970FB6F8949EBF0FBE8DBFEDB728
:10196000FEB7319680EB94E0ADB7BEB712969C936C
:101970008E93119783E091E09383828322573F4FA8
:10198000358324832F5F3F4F378326830E949D2911
:101990008DB79EB708960FB6F8949EBF0FBE8DBF49
:1019A0000895CF93DF93AC01E091EA04F091EB044A
:1019B00020913D0630913E06C9018C599F4F8E17EC
:1019C0009F071CF4EA01219709C024563040E21712
:1019D000F30714F0EA0102C0EA012196842F90E097
:1019E000C817D90729F088EA96E04C2F0E94553095
:1019F000CE01DF91CF9108950F931F9308EA16E06F
:101A0000C80163EF73E041E00E945530C80164EF04
:101A100073E043E10E945530C80165EF73E046E092
:101A20000E945530C80166EF73E040E10E945530D6
:101A3000C80167EF73E047E20E945530C80168EFC4
:101A400073E048E80E945530C80169EF73E043E154
:101A50000E9455301F910F910895CF92DF92EF921F
:101A6000FF920F931F937C01D62EC72E00EB14E03C
:101A7000C8016E2D4D2D0E946F04C8010E944705BC
:101A800000D000D0EDB7FEB71283018383E391E06D
:101A9000948383830E948C29EDB7FEB71283018360
:101AA00083E291E0948383830E948C29EDB7FEB793
:101AB0001283018383E191E0948383830E948C29C4
:101AC000EDB7FEB71283018383E091E094838383B3
:101AD0000E948C29EDB7FEB71283018384EF90E05A
:101AE000948383830E948C290F900F900F900F9006
:101AF000C8010E942B05C70101966D2D7C2D0E9407
:101B0000260B1F910F91FF90EF90DF90CF900895DB
:101B1000CF92DF92EF92FF920F931F93CF93DF93B9
:101B2000182F062F0E94363128EE33E040E050E0B7
:101B30000E94F13669017A01C0EBD4E0CE01612F39
:101B4000402F0E946F04CE010E9447058091060538
:101B500090910705892B09F453C000910805109155
:101B600009058DB79EB744970FB6F8949EBF0FBE78
:101B70008DBFEDB7FEB73196ADB7BEB71296DC9309
:101B8000CE93119788E091E09383828383EB90E07A
:101B900095838483C6016CE370E00E94DE36CB013E
:101BA0006CE370E00E94DE36978386832AE330E0A0
:101BB00031872087C6016CE370E00E94DE36938790
:101BC000828785E690E095878487C8016CE370E0A2
:101BD0000E94CA36CB016CE370E00E94DE36978724
:101BE0008687318B208BC8016CE370E00E94CA3677
:101BF000938B828B0E949D298DB79EB7449633C0EC
:101C0000ADB7BEB71C970FB6F894BEBF0FBEADBF41
:101C1000EDB7FEB731961296DC93CE93119780E222
:101C200091E09383828383EB90E095838483C60164
:101C30006CE370E00E94DE36CB016CE370E00E9442
:101C4000DE36978386838AE390E091878087C6019A
:101C50006CE370E00E94DE36938782870E949D29A4
:101C60008DB79EB70C960FB6F8949EBF0FBE8DBF72
:101C700080EB94E00E942B05DF91CF911F910F9193
:101C8000FF90EF90DF90CF900895EF92FF920F9327
:101C90001F93282F462FA0EBEA2EA4E0FA2EC701AF
:101CA000622F0E946F04C7010E9447058DB79EB73F
:101CB0000A970FB6F8949EBF0FBE8DBF0DB71EB723
:101CC0000F5F1F4FEDB7FEB7F282E1828CE291E029
:101CD000F8019383828360910A0570910B058091CE
:101CE0000C0590910D0520913406309135064091F8
:101CF0003606509137060E94A435F8016483758337
:101D00008683978380EB90E0918780870E949D294E
:101D10008DB79EB70A960FB6F8949EBF0FBE8DBFC3
:101D2000C7010E942B051F910F91FF90EF9008951E
:101D30008F929F92AF92BF92CF92DF92EF92FF92DB
:101D40000F931F93E82EF62E00EB14E0C8016E2DC2
:101D50004F2D0E946F04C8010E9447058DB79EB7A2
:101D60000C970FB6F8949EBF0FBE8DBFEDB7FEB7B0
:101D70003196ADB7BEB712961C930E93119794E3AC
:101D8000892E91E0992E938282828DEEA82EB12C1D
:101D9000B582A4828091130590911405A091150538
:101DA000B091160586839783A087B187B3EFCB2EBA
:101DB000D12CD386C2860E949D298DB79EB70C96E2
:101DC0000FB6F8949EBF0FBE8DBFC8010E942B05B1
:101DD000F394C8016E2D4F2D0E946F04C8010E941C
:101DE0004705ADB7BEB71C970FB6F894BEBF0FBE80
:101DF000ADBFEDB7FEB7319612961C930E931197B7
:101E000093828282B582A4828091170590911805F1
:101E1000A0911905B0911A0586839783A087B18791
:101E2000D386C2860E949D298DB79EB70C960FB6A9
:101E3000F8949EBF0FBE8DBFC8010E942B05F3947E
:101E4000C8016E2D4F2D0E946F04C8010E944705E6
:101E5000ADB7BEB71C970FB6F894BEBF0FBEADBFEF
:101E6000EDB7FEB7319612961C930E93119793829D
:101E70008282B582A48280911B0590911C05A0915D
:101E80001D05B0911E0586839783A087B187D386F1
:101E9000C2860E949D298DB79EB70C960FB6F89406
:101EA0009EBF0FBE8DBFC8010E942B051F910F91D1
:101EB000FF90EF90DF90CF90BF90AF909F908F906A
:101EC00008950F931F93282F462F00EB14E0C801AD
:101ED000622F0E946F04C8010E9447058DB79EB70C
:101EE0000A970FB6F8949EBF0FBE8DBFEDB7FEB731
:101EF0003196ADB7BEB712961C930E9311978EE331
:101F000091E09383828389EB90E095838483809131
:101F10000605909107059783868382E890E0918774
:101F200080870E949D298DB79EB70A960FB6F894B8
:101F30009EBF0FBE8DBFC8010E942B051F910F9140
:101F40000895EF92FF920F931F93282F462F30EBA7
:101F5000E32E34E0F32EC701622F0E946F04C70105
:101F60000E9447058DB79EB70C970FB6F8949EBF99
:101F70000FBE8DBF0DB71EB70F5F1F4FEDB7FEB77A
:101F8000F282E18286E491E0F8019383828384EE19
:101F900090E09583848360910405709105058827FE
:101FA00077FD8095982F0E9471342AE037ED43E247
:101FB0005CE30E94A435F80166837783808791876C
:101FC0008FE890E0938782870E949D298DB79EB706
:101FD0000C960FB6F8949EBF0FBE8DBFC7010E942E
:101FE0002B051F910F91FF90EF9008950F931F9372
:101FF000282F462F00EB14E0C801622F0E946F04C7
:10200000C8010E9447058DB79EB70C970FB6F8948C
:102010009EBF0FBE8DBFEDB7FEB73196ADB7BEB751
:1020200012961C930E93119786E491E0938382831A
:1020300082EE90E095838483809100059091010564
:10204000A0910205B091030586839783A087B1878D
:102050008EE890E0938782870E949D298DB79EB776
:102060000C960FB6F8949EBF0FBE8DBFC8010E949C
:102070002B051F910F9108950F931F93282F462F23
:1020800080EB94E0622F0E946F0480EB94E00E944A
:1020900047058091E704882319F420E531E057C013
:1020A000813019F424E531E052C0823019F428E57A
:1020B00031E04DC0833019F42CE531E048C0843064
:1020C00019F420E631E043C0853019F424E631E00C
:1020D0003EC0863019F428E631E039C0873019F463
:1020E0002CE631E034C0883019F420E731E02FC00D
:1020F000893019F424E731E02AC08A3019F428E73E
:1021000031E025C08B3019F42CE731E020C08C3051
:1021100019F420E831E01BC08D3019F424E831E0D7
:1021200016C08E3019F428E831E011C08F3019F450
:102130002CE831E00CC0803119F420E931E007C00F
:10214000813119F024E931E002C025E931E08DB791
:102150009EB708970FB6F8949EBF0FBE8DBFEDB720
:10216000FEB7319600EB14E0ADB7BEB712961C93E4
:102170000E93119789E991E09383828380EE90E03A
:1021800095838483378326830E949D298DB79EB7CC
:1021900008960FB6F8949EBF0FBE8DBFC8010E946F
:1021A0002B051F910F9108950F931F93282F462FF2
:1021B00000EB14E0C801622F0E946F04C8010E9466
:1021C00047058DB79EB70A970FB6F8949EBF0FBE0E
:1021D0008DBFEDB7FEB73196ADB7BEB712961C9363
:1021E0000E9311978EE991E09383828387E890E0C4
:1021F000958384838091E8049091E9049783868392
:1022000085E290E0918780870E949D298DB79EB7D7
:102210000A960FB6F8949EBF0FBE8DBFC8010E94EC
:102220002B051F910F9108950F931F93282F462F71
:1022300000EB14E0C801622F0E946F04C8010E94E5
:1022400047058DB79EB70A970FB6F8949EBF0FBE8D
:102250008DBFEDB7FEB73196ADB7BEB712961C93E2
:102260000E93119788EA91E0938382838091DA0438
:102270009091DB049583848380EB90E09783868341
:1022800081EB90E0918780870E949D298DB79EB752
:102290000A960FB6F8949EBF0FBE8DBFC8010E946C
:1022A0002B051F910F9108950F931F93282F462FF1
:1022B00000EB14E0C801622F0E946F04C8010E9465
:1022C00047058DB79EB70A970FB6F8949EBF0FBE0D
:1022D0008DBFEDB7FEB73196ADB7BEB712961C9362
:1022E0000E93119788EA91E0938382838091D804BA
:1022F0009091D9049583848380EB90E097838683C3
:1023000082EB90E0918780870E949D298DB79EB7D0
:102310000A960FB6F8949EBF0FBE8DBFC8010E94EB
:102320002B051F910F9108950F931F93282F462F70
:1023300000EB14E0C801622F0E946F04C8010E94E4
:1023400047058DB79EB70A970FB6F8949EBF0FBE8C
:102350008DBFEDB7FEB73196ADB7BEB712961C93E1
:102360000E93119780EB91E09383828381EE90E04E
:10237000958384838091B8029091B9029783868374
:1023800085E290E0918780870E949D298DB79EB756
:102390000A960FB6F8949EBF0FBE8DBFC8010E946B
:1023A0002B051F910F9108950F931F93282F462FF0
:1023B00000EB14E0C801622F0E946F04C8010E9464
:1023C00047058DB79EB70C970FB6F8949EBF0FBE0A
:1023D0008DBFEDB7FEB73196ADB7BEB712961C9361
:1023E0000E93119788EB91E09383828382EC91E0C6
:1023F0009583848380ED90E0978386838FE396E0D6
:102400009187808781ED90E0938782870E949D2944
:102410008DB79EB70C960FB6F8949EBF0FBE8DBFBA
:10242000C8010E942B051F910F9108950F931F93D0
:10243000282F462F00EB14E0C801622F0E946F0482
:10244000C8010E9447058DB79EB70A970FB6F8944A
:102450009EBF0FBE8DBFEDB7FEB73196ADB7BEB70D
:1024600012961C930E93119780ED91E093838283D3
:102470008091E2049091E304A091E404B091E5041A
:1024800084839583A683B78380EB90E091878087D0
:102490000E949D298DB79EB70A960FB6F8949EBFED
:1024A0000FBE8DBFC8010E942B051F910F9108958B
:1024B0000F931F93282F462F00EB14E0C801622FC3
:1024C0000E946F04C8010E9447058DB79EB70C9704
:1024D0000FB6F8949EBF0FBE8DBFEDB7FEB7319615
:1024E000ADB7BEB712961C930E93119788ED91E08D
:1024F0009383828386E190E0958384838091FC04BA
:102500009091FD04A091FE04B091FF04868397830F
:10251000A087B18788E890E0938782870E949D29F1
:102520008DB79EB70C960FB6F8949EBF0FBE8DBFA9
:10253000C8010E942B051F910F910895CF92DF9241
:10254000EF92FF920F931F93CF93DF93282F462F85
:10255000C0EBD4E0CE01622F0E946F04CE010E9436
:10256000470560914B0670914C0680914D06909105
:102570004E06209134063091350640913606509132
:1025800037060E94A4356B017C0120E030E04AE769
:1025900054E40E9499351816D4F58DB79EB70C9760
:1025A0000FB6F8949EBF0FBE8DBF0DB71EB70F5F5D
:1025B0001F4FADB7BEB71296DC93CE93119786E44A
:1025C00091E0F801938382838EEF90E0958384837A
:1025D0006091380670913906882777FD8095982F8D
:1025E0000E9471349B01AC01C701B6010E94D63331
:1025F000D80116966D937D938D939C931997809136
:102600003C061A968C931A971B961C9221C08DB784
:102610009EB70C970FB6F8949EBF0FBE8DBFEDB757
:10262000FEB73196ADB7BEB71296DC93CE93119735
:1026300082EE91E0938382838EEF90E09583848392
:10264000C682D782E086F18680913B068287138618
:102650000E949D29EDB7FEB73C960FB6F894FEBFD9
:102660000FBEEDBF80EB94E00E942B05DF91CF9170
:102670001F910F91FF90EF90DF90CF900895EF9210
:10268000FF920F931F93282F462F50EBE52E54E017
:10269000F52EC701622F0E946F04C7010E944705F3
:1026A0008DB79EB70C970FB6F8949EBF0FBE8DBF27
:1026B0000DB71EB70F5F1F4FEDB7FEB7F282E18275
:1026C00088ED91E0F8019383828389EE90E0958311
:1026D00084836091F8047091F9048091FA049091D8
:1026E000FB04209130063091310640913206509122
:1026F00033060E94A435F80166837783808791872B
:1027000080913A06828713860E949D298DB79EB7D5
:102710000C960FB6F8949EBF0FBE8DBFC7010E94E6
:102720002B051F910F91FF90EF900895EF92FF926C
:102730000F931F93282F462F60EBE62E64E0F62EB2
:10274000C701622F0E946F04C7010E9447058DB721
:102750009EB70C970FB6F8949EBF0FBE8DBF0DB7F6
:102760001EB70F5F1F4FEDB7FEB7F282E18282EE18
:1027700091E0F8019383828386EE90E095838483D1
:102780006091F4047091F5048091F6049091F7043F
:102790002091340630913506409136065091370627
:1027A0000E94A435F80166837783808791878091A2
:1027B0003B06828713860E949D298DB79EB70C9693
:1027C0000FB6F8949EBF0FBE8DBFC7010E942B05A8
:1027D0001F910F91FF90EF900895EF92FF920F934A
:1027E0001F93282F462F70EBE72E74E0F72EC701BA
:1027F000622F0E946F04C7010E9447058DB79EB7E4
:102800000C970FB6F8949EBF0FBE8DBF0DB71EB7C5
:102810000F5F1F4FEDB7FEB7F282E18282EE91E0CB
:10282000F8019383828387EE90E09583848360919F
:102830000E0570910F05882777FD8095982F0E94CF
:10284000713420913406309135064091360650910E
:1028500037060E94A435F8016683778380879187C5
:1028600080913B06828713860E949D298DB79EB773
:102870000C960FB6F8949EBF0FBE8DBFC7010E9485
:102880002B051F910F91FF90EF9008950F931F93C9
:10289000282F462F00EB14E0C801622F0E946F041E
:1028A000C8010E94470580914F060E94A00CC801F4
:1028B0000E942B051F910F910895EF92FF920F93A5
:1028C0001F93282F462FE0EBEE2EE4E0FE2EC701EB
:1028D000622F0E946F04C7010E9447058DB79EB703
:1028E0000C970FB6F8949EBF0FBE8DBF0DB71EB7E5
:1028F0000F5F1F4FEDB7FEB7F282E18282EE91E0EB
:10290000F801938382838FE190E0958384836091C3
:1029100050067091510680915206909153060E9484
:10292000713420913406309135064091360650912D
:1029300037060E94A435F8016683778380879187E4
:1029400080913B06828713860E949D298DB79EB792
:102950000C960FB6F8949EBF0FBE8DBFC7010E94A4
:102960002B051F910F91FF90EF9008950F931F93E8
:10297000282F462F00EB14E0C801622F0E946F043D
:10298000C8010E9447058DB79EB740970FB6F894CF
:102990009EBF0FBE8DBFEDB7FEB73196ADB7BEB7C8
:1029A00012961C930E9311978CEE91E09383828381
:1029B00083E890E0958384838091DE049091DF0426
:1029C000A091E004B091E10486839783A087B1874A
:1029D00084E890E0938782878091EE049091EF04E1
:1029E000A091F004B091F10484879587A687B787FA
:1029F0000E949D298DB79EB740960FB6F8949EBF52
:102A00000FBE8DBFC8010E942B051F910F91089525
:102A10000F931F93282F462F80EB94E0622F0E9484
:102A20006F0480EB94E00E9447058091F304282F07
:102A300030E0823030F4F4E0220F331FFA95E1F7F2
:102A400002C02150304000D000D000D0EDB7FEB71A
:102A5000319600EB14E0ADB7BEB712961C930E93FF
:102A6000119780E091E093838283358324830E94D1
:102A70009D298DB79EB706960FB6F8949EBF0FBEE0
:102A80008DBFC8010E942B051F910F9108950F93D0
:102A90001F93282F462F00EB14E0C801622F0E94DD
:102AA0006F04C8010E9447058DB79EB708970FB6FF
:102AB000F8949EBF0FBE8DBFEDB7FEB73196ADB790
:102AC000BEB712961C930E9311978EEF91E09383ED
:102AD00082838FE090E0958384838091F2048683E3
:102AE00017820E949D298DB79EB708960FB6F8945D
:102AF0009EBF0FBE8DBFC8010E942B051F910F9175
:102B000008950F931F9300EB14E0C80163E045E0C4
:102B10000E946F04C8010E94470500D000D0EDB7A5
:102B2000FEB7128301838DE591E0948383830E9435
:102B30008C29EDB7FEB71283018389E491E0948379
:102B400083830E948C29EDB7FEB71283018383E44F
:102B500091E0948383830E948C290F900F900F90B3
:102B60000F90C8010E942B051F910F9108950F939C
:102B70001F93282F462F00EB14E0C801622F0E94FC
:102B80006F04C8010E94470500D000D0EDB7FEB722
:102B90001283018384E791E0948383830E948C29CC
:102BA0000F900F900F900F90C8010E942B051F915E
:102BB0000F910895EF92FF920F931F93CF93DF939E
:102BC0000E9436312091590630915A0640915B0699
:102BD00050915C06261737074807590708F08AC145
:102BE0000E9436316C507E4F8F4F9F4F6093590635
:102BF00070935A0680935B0690935C0600EB14E09A
:102C0000C8010E949405C80165E043E00E946F047A
:102C1000C8010E94470500D000D0EDB7FEB712836F
:102C2000018384ED91E0948383830E948C290F902B
:102C30000F900F900F9080913D0690913E06892B4A
:102C400031F08091540690915506892B81F4809142
:102C5000EA049091EB0490933E0680933D068091A8
:102C6000EC049091ED0490935506809354062091C6
:102C7000EC043091ED044091540650915506C90181
:102C8000845690404817590724F4809158068F5F66
:102C900008C02C593F4F241735072CF48091580653
:102CA00081508093580680915806181614F081E0E0
:102CB00003C084301CF083E080935806809158064E
:102CC000823009F462C0833009F4BEC0813009F05B
:102CD0000DC100D000D0C0EBD4E0EDB7FEB7D28379
:102CE000C1838BEC91E0948383830E948C29809133
:102CF0002F060F900F900F900F9080FF22C000D0F2
:102D000000D0EDB7FEB7D283C18383EC91E094830A
:102D100083830E948C2980913D0690913E068456C3
:102D200090400F900F900F900F902091EA043091F7
:102D3000EB04281739070CF0D9C080912F068E7F3D
:102D400021C000D000D0EDB7FEB7D283C1838BEB9A
:102D500091E0948383830E948C2980913D06909119
:102D60003E068C599F4F0F900F900F900F9020911F
:102D7000EA043091EB04821793070CF0B7C08091FE
:102D80002F06816080932F06B1C000D000D0C0EB29
:102D9000D4E0EDB7FEB7D283C18381EB91E0948399
:102DA00083830E948C290F900F900F900F90809139
:102DB0005606882301F100D000D0EDB7FEB7D283CC
:102DC000C18387EA91E0948383830E948C29809158
:102DD0003D0690913E06845690400F900F900F90C4
:102DE0000F902091EA043091EB04281739071CF565
:102DF0001092560620C000D000D0EDB7FEB7D283A7
:102E0000C1838AE991E0948383830E948C29809115
:102E10003D0690913E068C599F4F0F900F900F905A
:102E20000F902091EA043091EB04821793071CF471
:102E300081E08093560688EA96E06BEF73E040915C
:102E400056060E94553052C000D000D0A0EBEA2EAA
:102E5000A4E0FA2EEDB7FEB7F282E18289E891E0B4
:102E6000948383830E948C298DB79EB708970FB6F1
:102E7000F8949EBF0FBE8DBF0DB71EB70F5F1F4FDB
:102E8000EDB7FEB7F282E18284E092E0F80193832D
:102E900082836091570670E080E090E00E946F347A
:102EA00020E030E040E251E40E94D633F801648330
:102EB00075838683978386E790E09187808780E299
:102EC00090E0938782870E949D298DB79EB70C96CC
:102ED0000FB6F8949EBF0FBE8DBF8091570690E04D
:102EE00060E873E00E94D10C8093570680EB94E079
:102EF0000E942B05DF91CF911F910F91FF90EF90D2
:102F000008952F923F924F925F926F927F928F928D
:102F10009F92AF92BF92CF92DF92EF92FF920F9368
:102F20001F93DF93CF93CDB7DEB72B970FB6F894EF
:102F3000DEBF0FBECDBF888769870E9436312091E2
:102F4000660630916706409168065091690626171B
:102F500037074807590708F069C180916A06882336
:102F6000C9F08093BA0210926A068CE092E09093C6
:102F70006C0680936B060E9436316C507E4F8F4FEB
:102F80009F4F6093660670936706809368069093E0
:102F9000690607C18091BA02282E33242091E604E5
:102FA0002F8300916B0610916C063091D304398306
:102FB0008091F3048E8390915D069D83E0902005BF
:102FC00060900005709001058090020590900305C7
:102FD000909157064090B8025090B90280915E06D9
:102FE000A82FB0E0BC83AB83B0915F06BA83F090AA
:102FF0001F053B862A86A92EBB24CC24DD24EA8526
:10300000FB853196FB87EA8737972CF021E030E08B
:103010003B872A871CC08A859B858330910539F1BF
:10302000843091053CF48130910589F0029709F0D4
:103030007FC015C0AA85BB85A530B10509F44EC077
:10304000A530B10504F1169709F072C058C0BF81D0
:10305000B23008F06DC009E112E081E070C0E98192
:10306000E33009F465C006E212E082E068C0FE8148
:10307000F23008F05DC02D81222309F459C003E32A
:1030800012E083E05CC031E03E1598F0C601B50166
:103090000E946F3420E030E040E251E40E94D633D9
:1030A0009B01AC01C401B3010E94CF3388230CF013
:1030B0003FC000E412E083E0E81649F094E0E9162E
:1030C00049F0A2E0EA1641F40DE412E005C00AE579
:1030D00012E002C007E612E084E031C0EB81FC811F
:1030E0004E165F062CF5FDE94F16FFEF5F0601F166
:1030F0002A812223E9F404E712E085E020C03F8121
:103100003230B0F481E08F1598F493E0F91649F06D
:10311000A4E0FA1649F0B2E0FB1651F401E812E01F
:1031200005C00DE812E002C00AE912E086E007C01F
:10313000EA85FB85E215F30509F061CF60C01093C5
:103140006C0600936B0680936A0681E080936006AC
:103150000E94363168517C4F8F4F9F4F60936606B7
:103160007093670680936806909369060E943631D3
:103170006056704F8F4F9F4F609362067093630647
:10318000809364069093650680916106882321F000
:1031900080EB94E00E9494051092610602C01092A8
:1031A000600600EB14E0C801688549850E946F0441
:1031B000C8010E94470500D000D000D0EDB7FEB78F
:1031C0003196ADB7BEB712961C930E93119787EA4E
:1031D00092E09383828380916B0690916C06958335
:1031E00084830E949D29EDB7FEB736960FB6F894FA
:1031F000FEBF0FBEEDBFC8010E942B0517C0109384
:103200006C0600936B0610926A060E94363120917C
:103210006206309163064091640650916506261758
:1032200037074807590708F4BACFBBCF2B960FB61C
:10323000F894DEBF0FBECDBFCF91DF911F910F91EC
:10324000FF90EF90DF90CF90BF90AF909F908F90C6
:103250007F906F905F904F903F902F900895EF92E6
:10326000FF920F931F9380916D06843009F056C032
:103270009091E704943008F027C180917606891771
:10328000A1F1909376060E94363160937206709396
:1032900073068093740690937506909176068091DC
:1032A000BB02981711F580916106813091F0813051
:1032B00018F08230B1F413C011E0109361060E943F
:1032C0003631615375478040904030F410936E065C
:1032D00008C082E08093610610926E0602C01092D0
:1032E000610680EB94E00E9494050E9436312091A3
:1032F0007206309173064091740650917506621BF8
:10330000730B840B950B615D77408040904008F40F
:10331000DBC08091E7048093BB02D6C0853029F4DE
:103320008091B0029091B10214C0863029F480914E
:10333000B2029091B3020DC0873029F48091B4029B
:103340009091B50206C0883041F48091B602909108
:10335000B702909371068093700680916F0620915A
:10336000700630917106882309F04AC0C90189505E
:1033700097408F5A9440C8F40E9436316153754784
:103380008040904020F481E080936E060CC08091D4
:103390006E06882341F480916006882321F480EB37
:1033A00094E00E94940582E028C044E0203B34076A
:1033B00068F480916106882349F010926E0680EBD4
:1033C00094E00E949405109261067EC0205B344018
:1033D0002955324008F078C080916106813009F4A7
:1033E00073C080916006882309F06EC010926E064B
:1033F00080EB94E00E94940581E08093610664C0B4
:10340000215B344008F460C00E9436316153754737
:103410008040904008F041C080916E068823E9F515
:10342000E0907206F0907306009174061091750694
:1034300088EE93E0A0E0B0E0E80EF91E0A1F1B1F23
:103440000E943631E616F70608071907E8F581E00D
:1034500080936E0617C010926E0680EB94E00E9477
:10346000940580916106823019F41092610603C0C0
:103470008F5F8093610680916106823018F082E050
:10348000809361060E9436316093720670937306D2
:10349000809374069093750617C0E0907206F090C2
:1034A0007306009174061091750688EE93E0A0E013
:1034B000B0E0E80EF91E0A1F1B1F0E943631E61607
:1034C000F7060807190738F21F910F91FF90EF9048
:1034D000089580916D06843010F00E942F1980911C
:1034E0006E06882319F00E94DA150895809113045E
:1034F00080FF08C0609179048091770490E070E0CB
:103500000E94811780916106823008F0FDC1A82FCA
:10351000B0E0FD01E35FFB4F808185FF0BC0FD0143
:10352000E75DFB4F6081A95DBB4F8C9190E070E03F
:103530000E94471580916106A82FB0E0FD01E35F6E
:10354000FB4F808186FF0BC0FD01E35DFB4F608177
:10355000A55DBB4F8C9190E070E00E9408158091B2
:103560005D06882309F43FC080916106A82FB0E072
:10357000FD01E35FFB4F808187FF0BC0FD01EF5C26
:10358000FB4F6081A15DBB4F8C9190E070E00E9489
:10359000B61480916106A82FB0E0FD01E15FFB4FFA
:1035A000808184FF0BC0FD01E75BFB4F6081A95B5D
:1035B000BB4F8C9190E070E00E945D148091610699
:1035C000A82FB0E0FD01E15FFB4F808183FF0BC0BE
:1035D000FD01EB5BFB4F6081AD5BBB4F8C9190E0DD
:1035E00070E00E94461480916106A82FB0E0FD01B2
:1035F000EF5EFB4F808187FF0BC0FD01EF59FB4F52
:103600006081A15ABB4F8C9190E070E00E94ED1355
:1036100080916106A82FB0E0FD01ED5EFB4F808137
:1036200083FF0BC0FD01EF57FB4F6081A158BB4FDB
:103630008C9190E070E00E94581280915D06882382
:1036400009F444C08091F304823008F43FC08091B3
:103650006106A82FB0E0FD01EB5EFB4F808182FF89
:103660000BC0FD01E357FB4F6081A557BB4F8C9109
:1036700090E070E00E949E1280916106A82FB0E059
:10368000FD01EF5EFB4F808182FF0BC0FD01E35A1D
:10369000FB4F6081A55ABB4F8C9190E070E00E9477
:1036A000961380916106A82FB0E0FD01EF5EFB4FFD
:1036B000808183FF0BC0FD01EB59FB4F6081AD5949
:1036C000BB4F8C9190E070E00E943F1380916106A7
:1036D000A82FB0E0FD01E15FFB4F808181FF0BC0AF
:1036E000FD01E35CFB4F6081A55CBB4F8C9190E0DA
:1036F00070E00E94161280916106A82FB0E0FD01D3
:10370000E15FFB4F808180FF0BC0FD01E75CFB4F59
:103710006081A95CBB4F8C9190E070E00E94D41155
:1037200080916106A82FB0E0FD01ED5EFB4F808126
:1037300086FF0BC0FD01E757FB4F6081A957BB4FC8
:103740008C9190E070E00E94941180916106A82F06
:10375000B0E0FD01E35FFB4F808182FF0BC0FD0104
:10376000EF5DFB4F6081A15EBB4F8C9190E070E0FC
:103770000E94541180916106A82FB0E0FD01E35F23
:10378000FB4F808181FF0BC0FD01E35EFB4F608139
:10379000A55EBB4F8C9190E070E00E941411809167
:1037A0006106A82FB0E0FD01EF5EFB4F808184FF32
:1037B0000BC0FD01E359FB4F6081A559BB4F8C91B4
:1037C00090E070E00E94D41080916106A82FB0E0D4
:1037D000FD01EF5EFB4F808185FF0BC0FD01EF58BF
:1037E000FB4F6081A159BB4F8C9190E070E00E942B
:1037F0003C1080916106A82FB0E0FD01E35FFB4F14
:10380000808183FF0BC0FD01EB5DFB4F6081AD5DEF
:10381000BB4F8C9190E070E00E94F60F80916106A2
:10382000A82FB0E0FD01EF5EFB4F808180FF0BC051
:10383000FD01E75AFB4F6081A95ABB4F8C9190E084
:1038400070E00E94A10F80916106A82FB0E0FD01F9
:10385000E35FFB4F808184FF0BC0FD01EB5CFB4FFE
:103860006081AD5CBB4F8C9190E070E00E94610F75
:1038700080916106A82FB0E0FD01EB5EFB4F8081D7
:1038800081FF18C080915606FD01E157FB4F813042
:1038900049F4AF56BB4F6C91808190E070E00E947C
:1038A000450E08C0AF56BB4F6C91808190E070E030
:1038B0000E94980E80916106A82FB0E0FD01E15FA3
:1038C000FB4F808187FF0BC0FD01EB5AFB4F6081EE
:1038D000AD5ABB4F8C9190E070E00E94880D8091B2
:1038E0006106A82FB0E0FD01EF5EFB4F808186FFEF
:1038F0000BC0FD01EB58FB4F6081AD58BB4F8C9165
:1039000090E070E00E942D0D089580EB94E00E94FD
:1039100094050E9481150E94060A0895CF93DF93B3
:10392000EC0180EB94E00E946B04C817D9073CF0CF
:1039300080EB94E00E946004892B09F42397CE0168
:10394000DF91CF910895EF92FF920F931F93CF9342
:10395000DF930091610610E08AEF90E0089F70010C
:10396000099FF00C189FF00C1124C7010E94EB0A6C
:10397000F801E35FFB4F882319F08081816002C06A
:1039800080818E7F808380916106C82FD0E0C7013F
:1039900002960E94EB0AC95EDB4F88838091610624
:1039A000C82FD0E0C70104960E94EB0A90E00E9465
:1039B0008E1CC75EDB4F88830091610610E0C70153
:1039C00088569F4F0E94EB0AF801E35FFB4F882364
:1039D00019F08081806102C080818F7E8083809118
:1039E0006106C82FD0E0C70186569F4F0E94EB0AA0
:1039F000CD5CDB4F888380916106C82FD0E0C70182
:103A000084569F4F0E94EB0A90E00E948E1CCB5C74
:103A1000DB4F88830091610610E0C70106960E9483
:103A2000EB0AF801E35FFB4F882319F08081826085
:103A300002C080818D7F808380916106C82FD0E095
:103A4000C70108960E94EB0AC55EDB4F8883809110
:103A50006106C82FD0E0C7010A960E94EB0A90E0E9
:103A60000E948E1CC35EDB4F88830091610610E0CC
:103A7000C7010C960E94EB0AF801E35FFB4F882315
:103A800019F08081846002C080818B7F8083809167
:103A90006106C82FD0E0C7010E960E94EB0AC15EF6
:103AA000DB4F888380916106C82FD0E0C701409624
:103AB0000E94EB0A90E00E948E1CCF5DDB4F888352
:103AC0000091610610E0C70142960E94EB0AF801DE
:103AD000E35FFB4F882319F08081886002C08081FA
:103AE000877F808380916106C82FD0E0C70144960C
:103AF0000E94EB0ACD5DDB4F888380916106C82F61
:103B0000D0E0C70146960E94EB0A90E00E948E1C0E
:103B1000CB5DDB4F88830091610610E0C7014E96B4
:103B20000E94EB0AF801E35FFB4F882319F08081C4
:103B3000806202C080818F7D808380916106C82F62
:103B4000D0E0C70180960E94EB0AC95DDB4F8883F5
:103B500080916106C82FD0E0C70182960E94EB0ACF
:103B600090E00E948E1CC75DDB4F88830091610648
:103B700010E0C70184960E94EB0AF801E35FFB4F57
:103B8000882319F08081806402C080818F7B8083CC
:103B900080916106C82FD0E0C70186960E94EB0A8B
:103BA000C55DDB4F888380916106C82FD0E0C701D7
:103BB00088960E94EB0A90E00E948E1CC35DDB4F4A
:103BC00088830091610610E0C7018A960E94EB0A83
:103BD000F801E35FFB4F882319F08081806802C001
:103BE00080818F77808380916106C82FD0E0C701E4
:103BF0008C960E94EB0AC15DDB4F88838091610641
:103C0000C82FD0E0C7018E960E94EB0A90E00E9478
:103C10008E1CCF5CDB4F88830091610610E0C701EA
:103C2000C0960E94EB0AF801E15FFB4F882319F070
:103C30008081816002C080818E7F80838091610657
:103C4000C82FD0E0C701C2960E94EB0AC95CDB4FC7
:103C5000888380916106C82FD0E0C701C4960E9476
:103C6000EB0A90E00E948E1CC75CDB4F88830091BA
:103C7000610610E0C701C6960E94EB0AF801E15FF9
:103C8000FB4F882319F08081826002C080818D7F84
:103C9000808380916106C82FD0E0C701C8960E943A
:103CA000EB0AC55CDB4F888380916106C82FD0E0AA
:103CB000C701CA960E94EB0A90E00E948E1CC35C6A
:103CC000DB4F88830091610610E0C701CC960E940B
:103CD000EB0AF801E15FFB4F882319F080818460D3
:103CE00002C080818B7F808380916106C82FD0E0E5
:103CF000C701CE960E94EB0AC15CDB4F888380919E
:103D00006106C82FD0E0C701805C9F4F0E94EB0A7C
:103D100090E00E948E1CCF5BDB4F88830091610690
:103D200010E0C701885B9F4F0E94EB0AF801E15F3A
:103D3000FB4F882319F08081806102C080818F7ED3
:103D4000808380916106C82FD0E0C701865B9F4FBA
:103D50000E94EB0AC95BDB4F888380916106C82F04
:103D6000D0E0C701845B9F4F0E94EB0A90E00E9465
:103D70008E1CC75BDB4F88830091610610E0C70192
:103D80008E5B9F4F0E94EB0AF801E15FFB4F882397
:103D900019F08081886002C08081877F8083809154
:103DA0006106C82FD0E0C7018C5B9F4F0E94EB0AD1
:103DB000CD5BDB4F888380916106C82FD0E0C701BF
:103DC0008A5B9F4F0E94EB0A90E00E948E1CCB5BA7
:103DD000DB4F88830091610610E0C701805B9F4F35
:103DE0000E94EB0AF801E15FFB4F882319F0808104
:103DF000806202C080818F7D808380916106C82FA0
:103E0000D0E0C7018E5A9F4F0E94EB0AC55BDB4F83
:103E1000888380916106C82FD0E0C7018C5A9F4FDC
:103E20000E94EB0A90E00E948E1CC35BDB4F8883EC
:103E30000091610610E0C7018A5A9F4F0E94EB0A69
:103E4000F801E15FFB4F882319F08081806402C094
:103E500080818F7B808380916106C82FD0E0C7016D
:103E6000885A9F4F0E94EB0AC15BDB4F8883809189
:103E70006106C82FD0E0C701865A9F4F0E94EB0A07
:103E800090E00E948E1CCF5ADB4F88830091610620
:103E900010E0C70182569F4F0E94EB0AF801E15FD4
:103EA000FB4F882319F08081806802C080818F7762
:103EB000808380916106C82FD0E0C70180569F4F54
:103EC0000E94EB0ACD5ADB4F888380916106C82F90
:103ED000D0E0C7018E559F4F0E94EB0A90E00E94F0
:103EE0008E1CCB5ADB4F88830091610610E0C7011E
:103EF0008E599F4F0E94EB0AF801EF5EFB4F88231B
:103F000019F08081816002C080818E7F80838091E2
:103F10006106C82FD0E0C7018C599F4F0E94EB0A61
:103F2000C95ADB4F888380916106C82FD0E0C70152
:103F30008A599F4F0E94EB0A90E00E948E1CC75A3C
:103F4000DB4F88830091610610E0C70182599F4FC3
:103F50000E94EB0AF801EF5EFB4F882319F0808185
:103F6000846002C080818B7F808380916106C82F2E
:103F7000D0E0C70180599F4F0E94EB0AC55ADB4F22
:103F8000888380916106C82FD0E0C7018E589F4F6B
:103F90000E94EB0A90E00E948E1CC35ADB4F88837C
:103FA0000091610610E0C70184579F4F0E94EB0A01
:103FB000F801EF5EFB4F882319F08081806802C012
:103FC00080818F77808380916106C82FD0E0C70100
:103FD00082579F4F0E94EB0AC15ADB4F8883809122
:103FE0006106C82FD0E0C70180579F4F0E94EB0A9F
:103FF00090E00E948E1CCF59DB4F888300916106B0
:1040000010E0C7018E569F4F0E94EB0AF801EF5E49
:10401000FB4F882319F08081826002C080818D7FF0
:10402000808380916106C82FD0E0C7018C569F4FD6
:104030000E94EB0AC959DB4F888380916106C82F23
:10404000D0E0C7018A569F4F0E94EB0A90E00E9481
:104050008E1CC759DB4F88830091610610E0C701B1
:104060008C589F4F0E94EB0AF801EF5EFB4F8823AC
:1040700019F08081886002C08081877F8083809171
:104080006106C82FD0E0C7018A589F4F0E94EB0AF3
:10409000CD59DB4F888380916106C82FD0E0C701DE
:1040A00088589F4F0E94EB0A90E00E948E1CCB59CB
:1040B000DB4F88830091610610E0C70186589F4F4F
:1040C0000E94EB0AF801EF5EFB4F882319F0808114
:1040D000806102C080818F7E808380916106C82FBD
:1040E000D0E0C70184589F4F0E94EB0AC559DB4FAF
:1040F000888380916106C82FD0E0C70182589F4F06
:104100000E94EB0A90E00E948E1CC359DB4F88830B
:104110000091610610E0C70180589F4F0E94EB0A92
:10412000F801EF5EFB4F882319F08081806202C0A6
:1041300080818F7D808380916106C82FD0E0C70188
:104140008E579F4F0E94EB0AC159DB4F88838091A5
:104150006106C82FD0E0C7018C579F4F0E94EB0A21
:1041600090E00E948E1CCF58DB4F8883009161063F
:1041700010E0C7018A579F4F0E94EB0AF801EF5EDB
:10418000FB4F882319F08081806402C080818F7B7F
:10419000808380916106C82FD0E0C70188579F4F68
:1041A0000E94EB0ACD58DB4F888380916106C82FAF
:1041B000D0E0C70186579F4F0E94EB0A90E00E9413
:1041C0008E1CCB58DB4F88830091610610E0C7013D
:1041D0008C559F4F0E94EB0AF801ED5EFB4F882340
:1041E00019F08081816002C080818E7F8083809100
:1041F0006106C82FD0E0C7018A559F4F0E94EB0A85
:10420000C958DB4F888380916106C82FD0E0C70171
:1042100088559F4F0E94EB0A90E00E948E1CC75861
:10422000DB4F88830091610610E0C70180559F4FE6
:104230000E94EB0AF801ED5EFB4F882319F08081A4
:10424000846002C080818B7F808380916106C82F4B
:10425000D0E0C7018E549F4F0E94EB0AC558DB4F38
:10426000888380916106C82FD0E0C7018C549F4F8E
:104270000E94EB0A90E00E948E1CC358DB4F88839B
:104280000091610610E0C7018A549F4F0E94EB0A1B
:10429000F801ED5EFB4F882319F08081886002C031
:1042A0008081877F808380916106C82FD0E0C7011D
:1042B00088549F4F0E94EB0AC158DB4F888380913E
:1042C0006106C82FD0E0C70186549F4F0E94EB0AB9
:1042D00090E00E948E1CCF57DB4F888300916106CF
:1042E00010E0C70184549F4F0E94EB0AF801ED5E75
:1042F000FB4F882319F08081806102C080818F7E0E
:10430000808380916106C82FD0E0C70182549F4FFF
:104310000E94EB0ACD57DB4F888380916106C82F3E
:10432000D0E0C70180549F4F0E94EB0A90E00E94AA
:104330008E1CCB57DB4F88830091610610E0C701CC
:10434000845A9F4F0E94EB0AF801ED5EFB4F8823D1
:1043500019F08081806402C080818F7B808380918E
:104360006106C82FD0E0C701825A9F4F0E94EB0A16
:10437000C957DB4F888380916106C82FD0E0C70101
:10438000805A9F4F0E94EB0A90E00E948E1CC757F4
:10439000DB4F88830091610610E0C70180529F4F78
:1043A0000E94EB0AF801EB5EFB4F882319F0808135
:1043B000846002C080818B7F808380916106C82FDA
:1043C000D0E0C7018E519F4F0E94EB0AC557DB4FCB
:1043D000888380916106C82FD0E0C7018C519F4F20
:1043E0000E94EB0A90E00E948E1CC357DB4F88832B
:1043F0000091610610E0C7018C529F4F0E94EB0AAA
:10440000F801EB5EFB4F882319F08081826002C0C7
:1044100080818D7F808380916106C82FD0E0C701A5
:104420008A529F4F0E94EB0AC157DB4F88838091CD
:104430006106C82FD0E0C70188529F4F0E94EB0A47
:1044400090E00E948E1CCF56DB4F8883DF91CF9186
:104450001F910F91FF90EF9008954F925F927F927E
:104460008F929F92AF92BF92CF92DF92EF92FF9284
:104470000F931F93DF93CF93CDB7DEB7C854D040CF
:104480000FB6F894DEBF0FBECDBF00EB14E0C8013D
:104490000E949405C80166E049E00E946F04C801CB
:1044A0000E94470500D000D0EDB7FEB7128301830C
:1044B0008FEF91E0948383830E948C290F900F905B
:1044C0000F900F90C8010E942B0500D000D003E987
:1044D00014E0EDB7FEB7128301838FEE91E0948371
:1044E00083830E948C2944EE442E41E0542EEE2416
:1044F000FF24CC24DD240F900F900F900F90702E8E
:10450000012F39E0A32EB12CAC0EBD1E4E01089434
:10451000811C911C83E994E00E94402A982F8D30E1
:1045200031F08D30DCF180538230C0F530C018306E
:10453000A1F59981892F8053823078F5913311F458
:1045400090E801C090E08A81813309F4905C8B810E
:10455000813309F4905E8C81813309F4905F8D8101
:10456000813309F4985F8E81813309F49C5F8F81D8
:10457000813309F49E5F8885813309F49F5FF501DB
:10458000EE0DFF1D90830894E11CF11C06C0F401A0
:10459000E10FF11D90831F5F01C010E0F0E4EF1602
:1045A000F104C9F480EB94E0B601A5010E947F04F8
:1045B0000894C11CD11C00D000D0EDB7FEB77182A9
:1045C0000283548243820E948C29EE24FF240F90A0
:1045D0000F900F900F90FFEFCF16D10409F00CF45D
:1045E00099CFC85BDF4F0FB6F894DEBF0FBECDBFCB
:1045F000CF91DF911F910F91FF90EF90DF90CF90BF
:10460000BF90AF909F908F907F905F904F90089554
:10461000DF92EF92FF920F931F93DF93CF93CDB76B
:10462000DEB72A970FB6F894DEBF0FBECDBF63E0AA
:10463000E62EF12CEC0EFD1E53E0D52EF6C30E94A3
:10464000363160527E4480409040C8F40E9436313A
:10465000695873418040904090F01A3011F01D303D
:1046600031F480912B068F5F80932B0602C010924D
:104670002B0680912B06833011F40E942D22812F6E
:1046800061E275E00E94F106882311F400E0C7C3DF
:104690008091250590912605A0912705B0912805C8
:1046A000863E46EA940746E2A4074DE7B40709F4BC
:1046B0008EC2873E56EA950756E2A5075DE7B50725
:1046C00008F0EFC08832EEE59E07E2EDAE07E4E2C7
:1046D000BE0709F427C28932FEE59F07F2EDAF0756
:1046E000F4E2BF0708F06AC088392CE292072AE199
:1046F000A20726E1B20709F41EC289393CE29307FA
:104700003AE1A30736E1B30740F586314AEA940758
:1047100047E3A4074BE0B40709F404C287315AEA1F
:10472000950757E3A5075BE0B50738F48E5F9B4C10
:10473000A74CB94009F069C360C38430FAE99F0708
:10474000F7EDAF07FEE0BF0709F4ECC18259934AC9
:10475000AC4EB44109F059C3E5C184373BEE930731
:104760003AE7A3073BE1B30709F4DCC185374BEE19
:1047700094074AE7A4074BE1B40780F480355FED66
:1047800095075DEEA50758E1B50709F40BC38E5CEC
:104790009844A745BA4109F038C319C28434FBEDE7
:1047A0009F07F0E7AF07FDE1BF0709F426C3825D6D
:1047B000924CA248BE4109F028C3BDC1883536EBF2
:1047C00093073DEFA3073AE4B30709F4CDC2893557
:1047D00046EB94074DEFA4074AE4B40788F5863EFC
:1047E00055ED95075AEDA50753E3B50709F448C100
:1047F000873EE5ED9E07EAEDAE07E3E3BE0780F4F2
:104800008E37F9EA9F07FBE5AF07F6E2BF0709F429
:1048100092C182559342A649B64209F0F6C254C2EB
:10482000883F3CEA93073EEEA30734E3B30709F45D
:10483000E4C2865A9E40A241B84409F0E6C27DC255
:1048400080365BED95075BE3A5075EE6B50709F4E7
:1048500069C18136EBED9E07EBE3AE07EEE6BE07DE
:1048600080F4823EF5E59F07FCE9AF07F6E6BF0757
:1048700009F48AC28C5E9943A647BB4609F0C5C2BB
:10488000BCC28A3B37EC930731E2A30734E7B30796
:1048900009F4F6C08A57974CA94DBB4709F0B5C239
:1048A000ACC28A3B54E8950755E2A5075EEBB50715
:1048B00009F46AC28B3BE4E89E07E5E2AE07EEEB43
:1048C000BE0708F06AC08E37F2E19F07FAE6AF072D
:1048D000FBE9BF0709F426C18F3722E192072AE6D8
:1048E000A2072BE9B20740F582353AEE930730E88C
:1048F000A3073AE8B30709F415C183354AEE9407D4
:1049000040E8A4074AE8B40738F486549340A24C20
:10491000B54809F07AC271C28C38E5E89E07E7EA2B
:10492000AE07E8E9BE0709F452C18A569E42A24684
:10493000B94909F06AC201C280322EE4920729EA1D
:10494000A20721EBB20709F41FC281323EE49307AC
:1049500039EAA30731EBB30780F48A3746EF9407AF
:1049600041EFA4074DE9B40709F431C18E5F964BBE
:10497000A942B54A09F049C22AC18A38E7EF9E0721
:10498000E7ECAE07E8EBBE0709F4D5C0845A9040C7
:10499000AB49BA4B09F039C230C2843629ED9207CF
:1049A00020EEA20727EDB20709F46AC0853639ED7B
:1049B000930730EEA30737EDB30788F586384BE34E
:1049C000940740EAA40744ECB40709F4DDC1873832
:1049D0005BE3950750EAA50754ECB50780F48C36E5
:1049E000E8E69E07E3E4AE07E2ECBE0709F45CC12B
:1049F00080589447A041B44C09F007C29CC084354C
:104A00002DE292072FEFA20725ECB20709F48AC026
:104A100086599543A840B24D09F0F7C155C18E346F
:104A20004DE594074EE3A40743EEB40709F47AC0BA
:104A30008F345DE595075EE3A50753EEB50780F477
:104A40008437E7E39E07E4EDAE07EEEDBE0709F419
:104A50009BC1865B9342A34AB24E09F0D6C1B7C050
:104A6000823920E7920726E8A2072BEFB20709F464
:104A7000C4C1825F9D4EA442BD4F09F0C6C18DC125
:104A80000E9436316093D4047093D5048093D60489
:104A90009093D704D092D30481E295E060E170E076
:104AA0000E94C5080E943E347093D9046093D804D4
:104AB00081E295E064E170E00E94C5080E943E3406
:104AC0007093DB046093DA0481E295E068E170E0C2
:104AD0000E94C5080E943E348B017093DD046093F0
:104AE000DC046091DE047091DF048091E004909119
:104AF000E10420E030E040E050E00E94CF33882322
:104B000079F4B801882777FD8095982F0E94713439
:104B10006093E2047093E3048093E4049093E504CB
:104B200001E074C180912B058093E60480912C05EF
:104B30008093E7046AC181E295E060E070E00E9442
:104B4000C50820E030E048EC52E40E94A4350E9401
:104B50003E347093E9046093E804693C710520F0E9
:104B60001092E9041092E804809145059091460561
:104B70009093EB048093EA04809147059091480557
:104B80009093ED048093EC0480914B0590914C053B
:104B90009093B1028093B00280914F05909150059F
:104BA0009093B3028093B202809151059091520587
:104BB0009093B5028093B40280915305909154056F
:104BC0009A8389839093B7028093B6021EC1609145
:104BD0002B0570912C0580912D0590912E050E943A
:104BE000713420E836E948E15BE40E94D6336093F3
:104BF000DE047093DF048093E0049093E1046091FD
:104C00002F05709130058091310590913205D701C3
:104C10006C9311967C93119712968C93129713961E
:104C20009C930E94713420E836E948E15BE40E94DD
:104C3000D6336093EE047093EF048093F004909366
:104C4000F104809150058093F20480914F05809388
:104C5000F30481E295E060E170E00E94C508609392
:104C6000E2047093E3048093E4049093E50481E20A
:104C700095E068E070E00E94C5086093F4047093CA
:104C8000F5048093F6049093F70481E295E064E1E3
:104C900070E00E94C5086093F8047093F904809353
:104CA000FA049093FB04B1C081E295E068E070E003
:104CB0000E94C50890586093FC047093FD04809393
:104CC000FE049093FF04A1C081E295E060E070E0F3
:104CD0000E94C5086093000570930105809302054A
:104CE0009093030581E295E064E070E00E94C508BE
:104CF00020E030E048EC52E40E94A4350E943E34AB
:104D0000709305056093040581E295E064E170E02D
:104D10000E94C5080E943E34709307056093060503
:104D200081E295E068E170E00E94C5080E943E348F
:104D3000709309056093080568C081E295E064E01E
:104D400070E00E94C5080E943E34882777FD809558
:104D5000982F0E94713460930A0570930B0580931D
:104D60000C0590930D0551C081E295E068E070E07C
:104D70000E94C5080E943E34709561957F4F7093E4
:104D80000F0560930E0541C080918B05809310053F
:104D900080918C058093110538C080912B058093FC
:104DA000120533C081E295E060E070E00E94C50822
:104DB0006093130570931405809315059093160561
:104DC00081E295E064E070E00E94C50860931705F9
:104DD000709318058093190590931A0581E295E068
:104DE00068E070E00E94C50860931B0570931C0585
:104DF00080931D0590931E0508C080913705809310
:104E00001F0580913C058093200500E080912205DC
:104E1000823229F481E295E063E20E94DD098EEBA3
:104E200090E00E949D31002331F583E994E00E94D7
:104E3000102A18161906F4F483E994E00E94402A17
:104E4000182F8091D304882309F019CCF8CB109245
:104E5000D30401E0802F90E02A960FB6F894DEBFCD
:104E60000FBECDBFCF91DF911F910F91FF90EF90BB
:104E7000DF90089500E02091D4043091D504409152
:104E8000D6045091D704205F384D4F4F5F4F2F838A
:104E9000388749875A870E9436312F81388549855E
:104EA0005A85261737074807590788F2D3CF1F932B
:104EB000CF93DF9385E090E06CE070E00E94B7153F
:104EC00068EE73E080E090E00E94443183E994E072
:104ED0000E948D2AC0E0D0E010E0CE016DE171E0CB
:104EE0000E94DE36892BA9F41F5E80EB94E0612FCF
:104EF0004CE00E946F0480EB94E00E94470580EB39
:104F000094E06EEE0E94770580EB94E00E942B0502
:104F1000105161E070E080E090E00E944431219601
:104F200087E0C13DD807C9F6DF91CF911F91089561
:104F300086E061E00E947B3208950F931F9386E024
:104F400061E00E943C3203E914E0C80140E051EE08
:104F500060E070E00E94AE291093AA060093A906B3
:104F60000E94982780EB94E00E94CD050E94851C4A
:104F700064EF71E080E090E00E94443183EF93E0C1
:104F80000E94EB0A813011F00E94FC0C0E945C0A26
:104F90001092610607C00E94A31C809161068F5F7A
:104FA00080936106809161068230A8F310926106B9
:104FB0000E94572782EC94E06CE679E224E630E028
:104FC00040E050E000E00E94613080EB94E00E94FD
:104FD000940582EC94E00E94C7301F910F910895D0
:104FE0002F923F924F925F926F927F928F929F92F9
:104FF000AF92BF92CF92DF92EF92FF920F931F93E7
:10500000DF93CF9300D000D0CDB7DEB780915D069F
:10501000882309F4E1C0E0908206F09083060091B5
:10502000840610918506C801B7019F7725E33AEF02
:105030004EE85CE30E94A4350E94D33369837A83EF
:105040008B839C83C801B7012091DE043091DF047B
:105050004091E0045091E1040E9408331B012C01AF
:105060009F7720EC3BE649ED57E40E94A4355B01B5
:105070006C016091860670918706809188069091F8
:1050800089062091EE043091EF044091F004509194
:10509000F1040E9408333B014C019F7720EC3BE672
:1050A00049ED57E40E94A43529813A814B815C8106
:1050B0000E94A4357B018C01C601B501A6019501B2
:1050C0000E94A4355B016C01C801B701A8019701DA
:1050D0000E94A4359B01AC01C601B5010E940933B1
:1050E0000E942B360E943E34609350067093510606
:1050F000809352069093530660E070E080E89FE34F
:1051000029813A814B815C810E94D6339B01AC019D
:10511000C201B1010E94A43597FA909497F8909437
:10512000A40193010E947C3320EE3EE245E652E466
:105130000E94A43520E030E044EB52E40E940933A1
:105140000E943E349B01AC0197FF04C028593E4F9A
:105150004F4F5F4FCA01B901645B7040804090407F
:1051600097FF06C0CA01B9016C547F4F8F4F9F4F04
:105170000E9471342091E2043091E3044091E404F0
:105180005091E5040E9408330E943E3497FF04C00A
:1051900068597E4F8F4F9F4F0E94713420E030E05E
:1051A00044EB53E40E94D63320E030E040E851E481
:1051B0000E94A4350E94073620E030E040E85FE31B
:1051C0000E9409330E94433460934F06613108F412
:1051D0006CC010924F0669C08091F304823008F4CD
:1051E00064C08091F204853008F45FC0A0908A0604
:1051F0008DE18A1508F459C0E090F404F090F504AC
:105200000091F6041091F70460918B0670918C0662
:1052100080918D0690918E06A80197010E94083317
:105220009F7720E030E040E05FE30E949935181658
:105230005CF410928A06E0928B06F0928C06009342
:105240008D0610938E0631C08A2D8F5F80938A065B
:105250008E3159F58091DE049091DF04A091E00435
:10526000B091E1048093820690938306A093840614
:10527000B09385068091EE049091EF04A091F00424
:10528000B091F1048093860690938706A0938806D8
:10529000B0938906E0928F06F092900600939106F3
:1052A0001093920681E080935D060F900F900F900F
:1052B0000F90CF91DF911F910F91FF90EF90DF90B2
:1052C000CF90BF90AF909F908F907F906F905F90A6
:1052D0004F903F902F900895809112058093B802CF
:1052E0001092B9020E944E080E94F10A80EB94E0ED
:1052F0000E94F0270E94691A08950E940823892BB2
:1053000019F00E946C29089582EC94E00E94AF305D
:1053100008958FEF9FE70895DF93CF93CDB7DEB762
:10532000FE0139968D819E8161E04F8158859F01F4
:105330000E942D2CCF91DF910895DF93CF93CDB7AD
:10534000DEB7FE0139968D819E8160E04F815885E0
:105350009F010E942D2CCF91DF9108950F931F93F1
:10536000DC01ED91FC910288F389E02D20E030E032
:1053700000E010E009951F910F9108958F92AF9270
:10538000CF92EF92FF920F931F93DF93CF93CDB7FE
:10539000DEB7FC011382128288EE93E0A0E0B0E059
:1053A00084839583A683B78386EF93E0918380837C
:1053B0005587448737872687118B008BF38AE28ACB
:1053C000C48AA58A868A70E0CB0123E0880F991FE2
:1053D0002A95E1F79C012956394F308F278B81564A
:1053E000994F928F818F81E090E002C0880F991FC2
:1053F0006A95E2F72091A706282B2093A706CF01F4
:1054000040E051EE60E070E00E94AE29CF91DF9164
:105410001F910F91FF90EF90CF90AF908F900895D4
:10542000FC01838D882319F42FEF3FEF0DC007880F
:10543000F08DE02D2081318182819381281B390BF1
:105440008481958128233923C9010895FC01838D26
:10545000882319F42FEF3FEF11C0018CF28DE02D5E
:105460002081318182819381281B390B20953095D1
:1054700084819581282339232F5F3F4FC9010895E7
:10548000FC01838D882361F0A789B08D2D913C911B
:10549000119712968D919C9113972817390721F433
:1054A0004FEF5FEFCA01089512968D919C9113976B
:1054B0001696ED91FC911797E80FF91F408112960F
:1054C0008D919C911397019614962D913C9115976F
:1054D0008223932313969C938E93129750E0E2CFEE
:1054E000FC01838D882351F00788F08DE02D208109
:1054F0003181828193812817390721F42FEF3FEF03
:10550000C9010895828193810680F781E02DE80F1B
:10551000F91F8081282F30E0F3CFDC015796ED9101
:10552000FC91589782819381918380835996ED9164
:10553000FC915A9780819181938382830895DC0145
:105540005B968C915B978823A9F15996ED91FC911C
:105550005A97208131812F5F3F4F84819581282385
:1055600039235C968C915C97882329F08281938102
:1055700028173907F9F08281938128173907D9F361
:10558000808191810680F781E02DE80FF91F60830B
:105590005996ED91FC915A97318320835296ED9163
:1055A000FC915397808156969C91892B808321E0B2
:1055B00030E002C020E030E0C9010895CF93DF93CE
:1055C000EC011B821A828A819B81998388831D82C8
:1055D0001C828E819F81009721F00E94C1031F824F
:1055E0001E82DF91CF9108950F931F938C01DC01F0
:1055F0005296ED91FC915397208156968C91569737
:1056000055969C915597892B809582238083579638
:105610008D919C9158970E94DE2AF801818D928D80
:105620000E94DE2AD8015B961C921F910F9108956B
:105630000F931F93CF93DF938C01FC01138212828F
:10564000828193819183808341E0A1E0B0E001C039
:105650004F5FFD01042E02C0EE0FFF1F0A94E2F718
:105660009B0182E06130780710F020E032E0E21721
:10567000F30770F3C1E0D0E002C0CC0FDD1F4A9504
:10568000E2F72197F801268137812115310541F094
:10569000848195818C179D0789F0C9010E94C103FF
:1056A000F801D583C483CE0101960E9417039C01A3
:1056B000F8019783868380E0232B09F081E0DF9156
:1056C000CF911F910F910895AF92BF92CF92DF9229
:1056D000EF92FF920F931F93CF93DF937C015A01B8
:1056E0006B01E901DC015B968C915B978823F1F0FB
:1056F0002115310539F45796ED91FC915897C481E5
:10570000D58121960115110549F4D7015996ED91DE
:10571000FC915A97048115810F5F1F4FD701ED91BE
:10572000FC910088F189E02DC7010995F70187896F
:10573000908D209711F4C0E8D0E0BE010E94182B94
:10574000882381F0D70159968D919C915A97011524
:10575000110511F400E110E0B8010E94182B882314
:1057600009F04DC0D701ED91FC910088F189E02D41
:10577000C701099567C0D7015096ED91FC915197EB
:10578000B0E0AB16B1EEBB06B0E0CB06B0E0DB0696
:1057900009F454C081E090E0D70154960C9002C007
:1057A000880F991F0A94E2F7808360E079E08DE327
:1057B00090E0A60195010E941337215030404040EF
:1057C0005040CA01B90122E030E040E050E00E94C0
:1057D0001337D7011C96ED91FC911D9730831E96CF
:1057E000ED91FC911F972083D7015296ED91FC918A
:1057F0005397808155969C91892B808323C0D70134
:105800005996ED91FC915A9713821282828193816D
:10581000918380835796ED91FC9158971382128261
:10582000828193819183808381E05B968C931A14AB
:105830001B041C041D040CF49ECFD6CF108220E163
:1058400030E0C7CFDF91CF911F910F91FF90EF9084
:10585000DF90CF90BF90AF9008952F923F924F92DC
:105860005F926F927F928F929F92AF92BF92CF92F0
:10587000DF92EF92FF920F931F93DF93CF93CDB7F9
:10588000DEB764970FB6F894DEBF0FBECDBF3C0104
:10589000688B5A8B498B69011C01AE014F5F5F4FCA
:1058A0005C8B4B8BE989FA89488940FD659140FF03
:1058B0006191FA8BE98B662309F4D7C3653249F409
:1058C00040FD859140FF8191FA8BE98B8532B1F4DF
:1058D0000CC06A3051F4D301ED91FC910190F0813C
:1058E000E02DC1016DE009956AE0D301ED91FC91D5
:1058F0000190F081E02DC1010995D4CF982F10E0DF
:10590000882499241032B0F49B3269F09C3228F438
:10591000903251F0933271F40BC09D3239F09033D4
:1059200049F4116028C01260146025C0186023C0BB
:10593000106121C017FD2BC0892F80538A3078F465
:1059400016FF06C0BAE09B9E902C1124980E13C03F
:10595000EAE08E9E802C1124880E10620CC09E32CC
:1059600021F416FD82C3106406C09C3611F4106841
:1059700002C0983661F4E989FA89488940FD959119
:1059800040FF9191FA8BE98B992309F0BBCF892FC6
:105990008554833020F4812F8061905E07C0892F69
:1059A0008556833008F0E6C1812F8F7E86FD02C0C8
:1059B00076E0972E6FE3F62EF822953619F450E430
:1059C000F52A07C0963619F480E8F82A02C091102B
:1059D0009A94F7FE0BC09BE3991520F427E05CE353
:1059E000B52E0DC0B92CB39427E009C0A7E0A915C6
:1059F00020F447E0942E27E001C0292DBB24F601B6
:105A00003496FD87EC87D6016D917D918D919C91A7
:105A1000AE014F5F5F4F0B2D0E943F026C01098169
:105A2000E02FF0E0FF87EE8700FF05C0FE85F3FD65
:105A300002C01DE209C0F1FE02C01BE205C0F2FC7B
:105A400002C010E001C010E28E859F858C709070BE
:105A5000892B09F444C0112311F483E001C084E0D0
:105A6000881510F088240EC0881AF3FC0BC0D301EF
:105A7000ED91FC910190F081E02DC10160E209956A
:105A80008A94A9F7112349F0D301ED91FC9101907B
:105A9000F081E02DC101612F0995BE85B3FF03C0E0
:105AA00008E013E012C00CE013E00FC0E114F104B1
:105AB00009F06052D301ED91FC910190F081E02D4D
:105AC000C10109950F5F1F4F05C0EF2CFF24B0E106
:105AD000EB22FF24F8016491662341F748C1F7FEE9
:105AE00013C0BC0CFE85F4FF04C08A81813309F425
:105AF000BA941B141CF0BB24B3942DC048E04B1582
:105B000050F538E0B32E27C0F6FC25C0892D90E073
:105B10008C159D054CF05CEFC5165FEFD50624F0A3
:105B200080E8F82A01C09A94992049F0E2E0F0E078
:105B3000EC0FFD1FE90DF11D80818033A1F3F7FE0D
:105B40000AC0B92CB394892D90E0C816D90614F078
:105B5000992401C09C18F7FC03C025E030E009C07F
:105B60001C141D041CF021E030E003C096012F5FDF
:105B70003F4F112311F02F5F3F4F992029F0892DBE
:105B800090E00196280F391F882D90E028173907DB
:105B900014F0882401C0821A4F2C5524C201897048
:105BA0009070892B59F00CC0D301ED91FC910190BC
:105BB000F081E02DC10160E209958A948820A1F767
:105BC000112349F0D301ED91FC910190F081E02D7A
:105BD000C101612F099543FE0BC00CC0D301ED91AB
:105BE000FC910190F081E02DC10160E309958A9458
:105BF0008820A1F7F7FE51C08601D7FE02C000E061
:105C000010E076010894E11CF11CE01AF10AE1E0D1
:105C1000F0E0EC0FFD1FEE0EFF1E26014B185108A1
:105C2000892D90E0AA24BB24A81AB90AFFEF0F3FE0
:105C30001F0749F4D301ED91FC910190F081E02D13
:105C4000C1016EE20995C016D10634F04016510626
:105C50001CF4F701608101C060E30150104008941A
:105C6000E11CF11C0A151B054CF0D301ED91FC91D0
:105C70000190F081E02DC1010995D8CF0C151D05CB
:105C800041F48A81863320F4853319F4BE85B4FF4C
:105C900061E3D301ED91FC9165C06A81613309F044
:105CA0000F7ED301ED91FC910190F081E02DC101B7
:105CB00009959920E1F0D301ED91FC910190F081DB
:105CC000E02DC1016EE2099512E0E1E0F0E0EC0F99
:105CD000FD1FE10FF11D60811F5FD301ED91FC916C
:105CE0000190F081E02DC10109959A9471F7D301DB
:105CF000ED91FC910190F081E02D44FC02C065E63D
:105D000001C065E4C1010995D7FC05C0C114D104E7
:105D100041F404FF06C0D094C194D108D3946DE23D
:105D200001C06BE2D301ED91FC910190F081E02D77
:105D3000C101099560E305C06F5FE6EFFFEFCE0E8E
:105D4000DF1EFAE0CF16D104BCF7D301ED91FC9130
:105D50000190F081E02DC1010995D301ED91FC91F5
:105D60006C2D605D0190F081E02DC1010995CC841E
:105D7000DD8478C1933631F0933799F0933509F08B
:105D800061C023C0F601808189835E010894A11C53
:105D9000B11C42E050E0C40ED51E21E0E22EF12CF1
:105DA00012C0D601AD90BC9016FD03C06FEF7FEF1F
:105DB00002C0692D70E0E2E0F0E0CE0EDF1EC5010A
:105DC0000E9424047C011F7713C0D601AD90BC90C3
:105DD00016FD03C06FEF7FEF02C0692D70E0E2E0B7
:105DE000F0E0CE0EDF1EC5010E9419047C01106890
:105DF00013FF0BC023C0D301ED91FC910190F08102
:105E0000E02DC10160E209958A94882D90E0E816A2
:105E1000F90688F313C0F50117FD659117FF61912D
:105E20005F01D301ED91FC910190F081E02DC10162
:105E3000099581108A940894E108F108E114F104AD
:105E400051F710C1943611F0993699F517FF0AC031
:105E5000F601208131814281538184E090E0C80EB7
:105E6000D91E0CC0D6018D919C919C01442737FD11
:105E70004095542FE2E0F0E0CE0EDF1E9FE6F92EB3
:105E8000F12257FF09C050954095309521953F4F1D
:105E90004F4F5F4FF0E8FF2ACA01B901AE014F5FD3
:105EA0005F4F2AE030E00E94E101E82E4B89E41ABE
:105EB00041C0953721F41F7E2AE030E01CC0197FD5
:105EC0009F3661F0903720F4983509F0CEC00FC0AE
:105ED000903739F0983709F0C8C004C028E030E0A6
:105EE0000AC0106114FD146020E130E004C014FD0C
:105EF000166020E132E017FF08C0D6016D917D9158
:105F00008D919C91E4E0F0E008C0D6018D919C91C8
:105F1000BC0180E090E0E2E0F0E0CE0EDF1EAE01DA
:105F20004F5F5F4F0E94E101E82EFB89EF1A8FE778
:105F3000F82EF122F6FE0BC04EEFF422E91438F4ED
:105F4000F4FE07C0F2FC05C05FEEF52202C01E2D74
:105F500001C0192DF4FE0DC0FE01EE0DF11D808172
:105F6000803319F489EEF82208C01F5FF2FE05C0E5
:105F700003C08F2D867809F01F5F0F2DF3FC18C02A
:105F8000F0FE13C0181510F09E2C0FC09E2C980C1C
:105F9000911A182D0AC0D301ED91FC910190F08166
:105FA000E02DC10160E209951F5F1815A0F304C040
:105FB000181510F4811A01C0882404FF17C0D301FA
:105FC000ED91FC910190F081E02DC10160E3099514
:105FD00002FF29C0D301ED91FC910190F081E02DE9
:105FE00001FD02C068E712C068E510C0802F867806
:105FF000D1F001FF02C06BE201C060E2F7FC6DE28C
:10600000D301ED91FC910190F081E02DC101099542
:106010000AC0D301ED91FC910190F081E02DC10106
:1060200060E309959A94E914A0F3EA94D301ED9101
:10603000FC91A1E0B0E0AC0FBD1FAE0DB11D019011
:10604000F081E02DC1016C910995EE2071F70AC035
:10605000D301ED91FC910190F081E02DC10160E24E
:1060600009958A948820A1F71DCC64960FB6F89400
:10607000DEBF0FBECDBFCF91DF911F910F91FF907B
:10608000EF90DF90CF90BF90AF909F908F907F90D8
:106090006F905F904F903F902F900895F999FECFA9
:1060A00072BD61BDF89A80B50895F999FECF1FBA07
:1060B00072BD61BD40BD0FB6F894FA9AF99A0FBE51
:1060C00008950F93FC016115710511F480E011C072
:1060D0002183328343835483728761870170000F69
:1060E000000F000F8081877F802B82608B7F8083F1
:1060F00081E00F910895CF93DF93EC010E94363138
:106100009B01AC018D819E81AF81B885281739072D
:106110004A075B0728F4888184FD02C060E00DC057
:1061200089819A81AB81BC81820F931FA41FB51F07
:106130008D839E83AF83B88761E0222757FD239527
:10614000332744275527922F91709295907F88810D
:106150008F7E892B8883862FDF91CF910895CF93EF
:10616000DF93EC01888182FF0FC0CE010E947B305B
:10617000882351F0E985FA85309709F009958881DF
:1061800083FF02C08B7F8883DF91CF910895CF93E7
:10619000DF93EC0189859A85892BE1F089819A81C9
:1061A000AB81BC810097A105B105A1F00E943631F9
:1061B00029813A814B815C81260F371F481F591F67
:1061C0002D833E834F835887888184608F7E8883A8
:1061D00081E001C080E0DF91CF9108951F920F927E
:1061E0000FB60F9211242F933F938F939F93AF93EA
:1061F000BF938091AF069091B006A091B106B09187
:10620000B2063091B3060196A11DB11D232F2D5F5B
:106210002D3720F02D570196A11DB11D2093B306F7
:106220008093AF069093B006A093B106B093B206E8
:106230008091AB069091AC06A091AD06B091AE06F0
:106240000196A11DB11D8093AB069093AC06A0935F
:10625000AD06B093AE06BF91AF919F918F913F91E4
:106260002F910F900FBE0F901F9018958FB7F89435
:106270002091AF063091B0064091B1065091B20620
:106280008FBFB901CA0108959B01AC017FB7F89493
:106290008091AB069091AC06A091AD06B091AE0690
:1062A00066B5A89B05C06F3F19F00196A11DB11DF1
:1062B0007FBFBA2FA92F982F8827860F911DA11D68
:1062C000B11D62E0880F991FAA1FBB1F6A95D1F705
:1062D000BC012DC0FFB7F8948091AB069091AC063D
:1062E000A091AD06B091AE06E6B5A89B05C0EF3F04
:1062F00019F00196A11DB11DFFBFBA2FA92F982F2C
:1063000088278E0F911DA11DB11DE2E0880F991FF6
:10631000AA1FBB1FEA95D1F7861B970B885E934097
:10632000C8F2215030404040504068517C4F211508
:1063300031054105510571F60895019739F0880F2F
:10634000991F880F991F02970197F1F70895789484
:1063500084B5826084BD84B5816084BD85B582606A
:1063600085BD85B5816085BDEEE6F0E08081816008
:106370008083E1E8F0E01082808182608083808108
:1063800081608083E0E8F0E0808181608083E1EBE0
:10639000F0E0808184608083E0EBF0E080818160C8
:1063A0008083EAE7F0E0808184608083808182607E
:1063B0008083808181608083808180688083109267
:1063C000C10008951F920F920FB60F9211242F93C0
:1063D0003F934F935F936F937F938F939F93AF936D
:1063E000BF93EF93FF938091B4069091B506892BEC
:1063F00029F0E091B406F091B5060995FF91EF916F
:10640000BF91AF919F918F917F916F915F914F91CC
:106410003F912F910F900FBE0F901F9018951F92D4
:106420000F920FB60F9211242F933F934F935F93C8
:106430006F937F938F939F93AF93BF93EF93FF934C
:106440008091B6069091B706892B29F0E091B606A7
:10645000F091B7060995FF91EF91BF91AF919F9190
:106460008F917F916F915F914F913F912F910F90FD
:106470000FBE0F901F901895CF93DF93482F50E0D9
:10648000CA018E5B9C4FFC013491425D5C4FFA0166
:106490008491882369F190E0880F991FFC01E05FE7
:1064A000FC4FA591B491FC01E65EFC4FC591D491DF
:1064B000662351F42FB7F8948C91932F90958923EC
:1064C0008C93888189230BC0623061F42FB7F894D4
:1064D0008C91932F909589238C938881832B88832B
:1064E0002FBF06C09FB7F8948C91832B8C939FBFCE
:1064F000DF91CF910895482F50E0CA018A5A9C4FEE
:10650000FC012491CA018E5B9C4FFC019491425D79
:106510005C4FFA013491332309F440C0222351F136
:10652000233071F0243028F42130A1F0223011F50D
:1065300014C02630B1F02730C1F02430D9F404C0A3
:10654000809180008F7703C0809180008F7D809341
:10655000800010C084B58F7702C084B58F7D84BD64
:1065600009C08091B0008F7703C08091B0008F7D0B
:106570008093B000E32FF0E0EE0FFF1FE65EFC4FCC
:10658000A591B4912FB7F894662321F48C9190953E
:10659000892302C08C91892B8C932FBF0895CF92B1
:1065A000DF92EF92FF920F931F93CF93DF937C01C3
:1065B0006B018A01C0E0D0E00FC0D6016D916D0182
:1065C000D701ED91FC910190F081E02DC701099573
:1065D000C80FD91F015010400115110571F7CE01E8
:1065E000DF91CF911F910F91FF90EF90DF90CF90AF
:1065F0000895CF93DF930E94A7310E949D27C0E0AA
:10660000D0E00E947D292097E1F30E940000F9CF9D
:106610005058BB27AA270ED041C201D230F006D273
:1066200020F031F49F3F11F41EF4C0C10EF4E09548
:10663000E7FBB6C1E92F54D280F3BA17620773079C
:106640008407950718F071F49EF56CC20EF4E0957E
:106650000B2EBA2FA02D0B01B90190010C01CA011C
:10666000A0011124FF27591B99F0593F50F4503EC7
:1066700068F11A16F040A22F232F342F4427585FB9
:10668000F3CF469537952795A795F0405395C9F7D1
:106690007EF41F16BA0B620B730B840BBAF0915089
:1066A000A1F0FF0FBB1F661F771F881FC2F70EC028
:1066B000BA0F621F731F841F48F4879577956795FB
:1066C000B795F7959E3F08F0B3CF9395880F08F0E4
:1066D0009927EE0F979587950895A1D158F080E8F6
:1066E00091E009F49EEFA2D128F040E851E059F47E
:1066F0005EEF09C05BC116C2E92FE078F1D168F303
:10670000092E052AC1F3261737074807590738F01D
:106710000E2E07F8E02569F0E025E0640AC0EF637B
:1067200007F8009407FADB01B9019D01DC01CA01F9
:10673000AD01EF934AD0B2D10AD05F91552331F029
:106740002BED3FE049E450FD49EC63CF0895DF9322
:10675000DD27B92FBF7740E85FE316161706480715
:106760005B0710F4D92FE9D19F938F937F936F9399
:10677000BCD2E8E6F0E01DD191D12F913F914F912D
:106780005F91EED1DD2349F09058A2EA2AED3FE077
:1067900049EC5FE3D0785D274DDFDF917FC1DCD02E
:1067A00008F481E008954AD1E39589C10CD076C1FF
:1067B0003DD140F034D130F021F45F3F19F0F0C00A
:1067C0005111B1C1F3C08CD198F39923C9F355236A
:1067D000B1F3951B550BBB27AA27621773078407D4
:1067E00038F09F5F5F4F220F331F441FAA1FA9F38A
:1067F00033D00E2E3AF0E0E830D091505040E6957C
:10680000001CCAF729D0FE2F27D0660F771F881FDC
:10681000BB1F261737074807AB07B0E809F0BB0BCB
:10682000802DBF01FF2793585F4F2AF09E3F5105EF
:1068300068F0B6C078C15F3FECF3983EDCF3869514
:1068400077956795B795F7959F5FC9F7880F911D65
:106850009695879597F90895E1E0660F771F881F51
:10686000BB1F621773078407BA0720F0621B730B04
:10687000840BBA0BEE1F88F7E095089504D0689456
:10688000B11151C1089534D188F09F5790F0B92FBC
:106890009927B751A0F0D1F0660F771F881F991F75
:1068A0001AF0BA95C9F712C0B13081F03BD1B1E00E
:1068B000089538C1672F782F8827B85F39F0B93F1E
:1068C000CCF3869577956795B395D9F73EF4909577
:1068D0008095709561957F4F8F4F9F4F0895E894F5
:1068E00009C097FB3EF490958095709561957F4F18
:1068F0008F4F9F4F9923A9F0F92F96E9BB279395C6
:10690000F695879577956795B795F111F8CFFAF4D5
:10691000BB0F11F460FF1BC06F5F7F4F8F4F9F4F06
:1069200016C0882311F096E911C0772321F09EE864
:10693000872F762F05C0662371F096E8862F70E0CA
:1069400060E02AF09A95660F771F881FDAF7880FA4
:106950009695879597F90895990F0008550FAA0BFA
:10696000E0E8FEEF16161706E807F907C0F0121662
:106970001306E407F50798F0621B730B840B950B65
:1069800039F40A2661F0232B242B252B21F40895BA
:106990000A2609F4A140A6958FEF811D811D089557
:1069A00097F99F6780E870E060E008959FEF80ECC2
:1069B0000895DF93CF931F930F93FF92EF92DF928F
:1069C0007B018C01689405C0DA2EEF01C9D0FE016D
:1069D000E894A5912591359145915591AEF3EF013C
:1069E00029DEFE019701A801DA9479F7DF90EF9094
:1069F000FF900F911F91CF91DF9108959F938F93F7
:106A00007F936F93FF93EF939B01AC019DD0EF9128
:106A1000FF91CFDF2F913F914F915F9195C000245F
:106A20000A941616170618060906089500240A94F3
:106A300012161306140605060895B8CF59D0E8F3C8
:106A4000E894EFEFBB273FE048EC5FE76B3D73074F
:106A50008407950708F1FF279F57B25A6A4D7F4078
:106A6000894CF04032F4BE556542704F8643FF4F6B
:106A70000894EE1F915030F0BB0F661F771F881FE0
:106A8000FF1FEBCF9EE7882332F0BB0F661F771FF7
:106A9000881F9A95C1F79395E09565C1092E0394D7
:106AA000000C11F4882352F0BB0F40F4BF2B11F4FB
:106AB00060FF04C06F5F7F4F8F4F9F4F0895EF932C
:106AC000E0FF06C0A2EA2AED3FE049EC5FEBB2DD51
:106AD000E5DF0F90039401FC9058E5E9F0E08ECFDC
:106AE00057FD9058440F551F59F05F3F71F047957F
:106AF000880F97FB991F61F09F3F79F08795089564
:106B0000121613061406551FF2CF4695F1DF08C082
:106B1000161617061806991FF1CF8695710561059F
:106B200008940895E894BB2766277727CB0197F947
:106B3000089512DF08F48FEF08959B01AC0160E027
:106B400070E080E89FE332CE0BD0A8CF68DF28F05A
:106B50006DDF18F0952309F023CF28CF1124E3CF60
:106B6000BFDFA0F3959FD1F3950F50E0551F629FB3
:106B7000F001729FBB27F00DB11D639FAA27F00D96
:106B8000B11DAA1F649F6627B00DA11D661F829FBD
:106B90002227B00DA11D621F739FB00DA11D621FA2
:106BA000839FA00D611D221F749F3327A00D611DBF
:106BB000231F849F600D211D822F762F6A2F1124A1
:106BC0009F5750408AF0E1F088234AF0EE0FFF1FF4
:106BD000BB1F661F771F881F91505040A9F79E3F2B
:106BE000510570F0DDCE9FCF5F3FECF3983EDCF3B4
:106BF000869577956795B795F795E7959F5FC1F768
:106C0000FE2B880F911D9695879597F9089570DF53
:106C1000E0F09E37D8F09639B8F49E3848F4672FE4
:106C2000782F8827985FF9CF869577956795939504
:106C30009539D0F3B62FB1706B0F711D811D20F403
:106C4000879577956795939573C08DC06CCF11F438
:106C50000EF4ACCE88C04CDFD0F39923D9F3CEF339
:106C60009F57550B87FF8FD056959795B0E020F42E
:106C7000660F771F881FBB1F1F930F93002490017F
:106C8000A0018001F001A0E80E0F1F1F0A1E511D78
:106C9000601B710B8009B50B48F4600F711F801DDC
:106CA000B51F0E1B1F0B0A0A510907C02E0F3F1FED
:106CB0004A1F0E0F1F1F0A1E511D660F771F881FC8
:106CC000BB1FA695F795E795F8F606171707080670
:106CD0005B07211D311D411D0F911F91B901842FAB
:106CE0009158880F9695879508959B01AC012CCFFC
:106CF000DF93D92FA3DEE695D7952AED3FE049E44F
:106D00005FE3B33A6207730784079507D7952AF0C4
:106D1000A2EA49EC90688EDCC1DEE3EBF0E06EDEC7
:106D2000DD0F0BF00ADFDD0F0BF49058DF910895B3
:106D3000882371F4772321F09850872B762F07C092
:106D4000662311F499270DC09051862B70E060E006
:106D50002AF09A95660F771F881FDAF7880F9695A5
:106D6000879597F908959F3F49F0915028F48695AB
:106D700077956795B7959F5F80389F4F880F969559
:106D8000879597F9089591505040660F771F881F97
:106D9000D2F70895AA1BBB1B51E107C0AA1FBB1F56
:106DA000A617B70710F0A61BB70B881F991F5A9597
:106DB000A9F780959095BC01CD01089597FB092E08
:106DC00007260AD077FD04D0E5DF06D000201AF4AC
:106DD000709561957F4F0895F6F7909581959F4F37
:106DE0000895A1E21A2EAA1BBB1BFD010DC0AA1F0C
:106DF000BB1FEE1FFF1FA217B307E407F50720F024
:106E0000A21BB30BE40BF50B661F771F881F991F9E
:106E10001A9469F760957095809590959B01AC01E7
:106E2000BD01CF01089597FB092E05260ED057FD11
:106E300004D0D7DF0AD0001C38F450954095309527
:106E400021953F4F4F4F5F4F0895F6F790958095EE
:106E5000709561957F4F8F4F9F4F0895EE0FFF1FE5
:0C6E60000590F491E02D0994F894FFCF08
:106E6C002563002563256300256325326925632589
:106E7C003032697C256325326925632530326900FF
:106E8C0025632532692563253032690025352E307E
:106E9C0066256300256325312E3566256300256341
:106EAC00253569256300256325352E32662563005B
:106EBC006D616E007374310073743200737433003F
:106ECC00737434007374350073743600706820006A
:106EDC00636C200076722000686C200061702000CA
:106EEC00727462006C616E0070702000706F6900CB
:106EFC006163200000617420002563257300256305
:106F0C0025332E30692563002534692563256300FC
:106F1C00256325336925630025737C25632573253B
:106F2C00630020C0C0C0C0C0C7C0C0C0C0C020006B
:106F3C0025342E3066256300256325332E306625D7
:106F4C006300256325352E306625630025632531C6
:106F5C00312E36667C25632531312E36660025634D
:106F6C002532690025332E31662563002020202030
:106F7C0020202020202020200020206469736172B2
:106F8C006D6564202000206E6F2074656C20636F2B
:106F9C006D2000206E6F206770732066697820006A
:106FAC00202062617474206C6F7720200062617401
:106FBC0074207761726E696E6700626174746372BB
:106FCC0069746963616C002062617474206572720B
:106FDC006F7220006C696E6B207175616C697479CD
:106FEC00006D6167207761726E696E67006D616715
:106FFC0020637269746963616C00206D6167202085
:10700C006572726F7220002573002000BC060000B0
:10701C00E803E803E803E8039DFF016400000000B7
:10702C007705CF32750478047B047E048929000728
:10703C000E091C1B1215383F363124232A2D70776C
:10704C007E796C6B6265484F464154535A5DE0E75C
:10705C00EEE9FCFBF2F5D8DFD6D1C4C3CACD9097CC
:10706C009E998C8B8285A8AFA6A1B4B3BABDC7C0BC
:10707C00C9CEDBDCD5D2FFF8F1F6E3E4EDEAB7B02C
:10708C00B9BEABACA5A28F88818693949D9A27201C
:10709C00292E3B3C35321F18111603040D0A57508C
:1070AC00595E4B4C45426F68616673747D7A898E6C
:1070BC00878095929B9CB1B6BFB8ADAAA3A4F9FEEC
:1070CC00F7F0E5E2EBECC1C6CFC8DDDAD3D4696EDC
:1070DC00676075727B7C51565F584D4A4344191E4C
:1070EC00171005020B0C21262F283D3A33344E493C
:1070FC00404752555C5B7671787F6A6D64633E39AC
:10710C00303722252C2B0601080F1A1D1413AEA99B
:10711C00A0A7B2B5BCBB9691989F8A8D8483DED90B
:10712C00D0D7C2C5CCCBE6E1E8EFFAFDF4F3C2C090
:10713C00C0C1C0C0C1C0C0C4C0C0C1C0C0C1C0C03B
:10714C00C3C0C0C1C0C0C1C0C0C5C0C0C1C0C0C127
:10715C00C0C0000000009F2ACF32102A402A702A9B
:0A716C008D2A262AAE29F42A642B8E
:00000001FF
